:020000040000FA
:100000005DEF06F01200FFFF04EF10F01200FFFF9B
:10001000FFFFFFFFFFFFFFFF0CEF10F01200FFFFDD
:10002000FFFFFFFFFFFFFFFFFFFF00006C500CE131
:100030006896040100513C0BE842E8420D0802E1D9
:100040000ED801D046D808D0040E6C5C03E1689647
:1000500050D802D0000E02D0010E00D01200D9CF2D
:10006000E6FFE1CFD9FFE652040104BF046B0001B3
:10007000B76BAF6BB06BB56BB66B15EC04F0DF6AAA
:10008000DF50206E216A010E205C000E21581BE219
:100090000001B05101E017D0F76ADF34FE0BF736EC
:1000A000F66E740EF6260A0EF7220900F5CF20F040
:1000B0000800F5CF21F004D021C0FAFF2050F96EDE
:1000C000FBDFDF2ADDD7EED8E552E552E7CFD9FFD7
:1000D0001200020E0001AF5D0AE1A7D8040100BDC5
:1000E00003D0C80E006F02D0880E006F01D020D957
:1000F0001200040E0001B85D0AE112C46EFF6E50DA
:10010000000803E2050EB86F02D0030EB86F0001BD
:10011000AF0512E113D8020E0001B75D04E104013E
:10012000840E046F08D0040104BD03D0C80E046F10
:1001300002D0880E046F01D0FBD81200D9CFE6FFA1
:10014000E1CFD9FF020EE1260001080EB55D000ED9
:10015000B6590EE2B5C0DEFFB6C0DDFFB75103E110
:10016000010EB76F04D0B70502E1020EB76F03D0DE
:10017000080EDE6EDD6A040104930491010EDB506B
:100180000413DFCF05F4000EDB500001B55F010E54
:10019000DB50B65B180EB36F040EB46F0001B9A349
:1001A0001ED0D9CFE9FFDACFEAFFEE50ED1016E00E
:1001B000B1C0F6FFB2C0F7FF0800F550B3C0E9FFC9
:1001C000B4C0EAFFEF6E0001B32B000EB423B12BD5
:1001D000B223DF06010E01E2DB06E3D71CD0D9CF44
:1001E000E9FFDACFEAFFEE50ED1015E0B1C0E9FF0C
:1001F000B2C0EAFFEF50B3C0E9FFB4C0EAFFEF6E50
:100200000001B32B000EB423B12BB223DF06010E85
:1002100001E2DB06E4D7020EE15C02E2E16AE552AC
:10022000E16EE552E7CFD9FF1200D9CFE6FFE1CF6B
:10023000D9FF020EE126030E04010015E76E010E40
:10024000E7CFDBFF01C4DFFFDE500001B527DD5043
:10025000B623180EB16F040EB26FD9CFE9FFDACF13
:10026000EAFFEE50ED1014E0B1C0E9FFB2C0EAFFC2
:10027000EF50B3C0E9FFB4C0EAFFEF6EB32B000E3E
:10028000B423B12BB223DF06010E01E2DB06E5D772
:10029000020EE15C02E2E16AE552E16EE552E7CF6F
:1002A000D9FF12006D980001B0510CE10401080E55
:1002B000016F100E026F040E036F840E006F0401B5
:1002C000046F35D0040110AF22D00001B5510401F4
:1002D000165D0001B6510401175904E216C4B5F0C9
:1002E00017C4B6F02BDF0001010EAF6F0401080E3A
:1002F000016F100E026F040E036F800E006F040179
:10030000180E066F040E076FC80E046F10D00001A0
:10031000020EAF6F0401056BC80E046F0401080ED6
:10032000016F180E026F040E036FC80E006F1200EB
:100330000001AF6B0401080E016F100E026F040E76
:10034000036F8C0E006F0401046B1200550EA76E34
:10035000AA0EA76EA68212000001420E6A6F020E5C
:100360006B6F010E6C6F12000001606B6651605D77
:100370001EE260C020F0216A226A67512024F36ED9
:1003800068512120F46E69512220F86EF4CFF7FFF6
:10039000F3CFF6FF0800F5CF61F06051EA6A6A0F0B
:1003A000E96E000EEA2261C0EFFF602BDFD7F86A2A
:1003B0001200840EA66E0001606B6651605D27E23C
:1003C0006051EA6A6A0FE96E000EEA22EFCF23F06D
:1003D00060C020F0216A226A67512024F36E6851C0
:1003E0002120F46E69512220F86EF4CFF7FFF3CF8D
:1003F000F6FF23C0F5FF0C001F0E60151F0803E079
:100400006605605D01E1A2DF0001602BD6D7120016
:100410000001606B6651605D20E2940EA66E605133
:10042000206E216A060ED89020362136E804FBE1C2
:10043000226A21BE2268000167512024F36E6851B0
:100440002120F46E69512220F86EF4CFF7FFF3CF2C
:10045000F6FF7CDF0001602BDDD7F86A1200A66A88
:100460000001606B6651605D0EE267516025A96E08
:10047000A6806051EA6A6A0FE96E000EEA22A8CFF0
:10048000EFFF602BEFD712000001606B6651605DDB
:1004900013E267516025A96E6051EA6A6A0FE96E3E
:1004A000000EEA22EF50A86E040EA66E4FDFA6B231
:1004B000FED70001602BEAD71200C40EA66E000121
:1004C000606B6651605D20E26051EA6A6A0FE96E16
:1004D000000EEA22EFCF23F060C020F0216A226AEA
:1004E00067512024F36E68512120F46E6951222057
:1004F000F86EF4CFF7FFF3CFF6FF23C0F5FF0C0043
:1005000025DF0001602BDDD7F86A1200400EE66E91
:10051000650EE66E000EE66ED5EC03F0E552E55290
:10052000E552000870E20001606B00016551FF0AAE
:1005300057E0FA0A50E0010A3BE0070A34E0010AFA
:100540002DE0030A18E0070A16E0700A01E05AD00D
:1005500003DF0001040E606F04010CBFFDD7400EE5
:10056000E66E650EE66E000EE66E9BEC03F0E5525D
:10057000E552E55248D0F8DE050E0001602704017F
:100580000CBFFDD7400EE66E650EE66E000EE66E01
:100590009BEC03F0E552E552E55235D00ADF00014D
:1005A000010E606F30D034DF0001010E606F2BD080
:1005B00056DF050E0001602704010CBFFDD7400E79
:1005C000E66E650EE66E000EE66E9BEC03F0E552FD
:1005D000E552E55218D058DF0001010E606F13D0CC
:1005E00046EC05F00001636B646B00016307000ECD
:1005F000645B00016351641103E000000000F5D763
:10060000FF0001D000D01200040110511F0B01089F
:1006100001E079D0145101E076D0060E115D2EE193
:100620001351230A28E0010A13E0030A01E024D051
:100630000001020EB06F0001BA0505E10001960E3F
:10064000B16F090EB26F090E0001B56FB66B14D011
:100650000001020EB06F0001BA0505E100014D0E68
:10066000B16F0A0EB26F0001BA0504E11D0E000160
:10067000B56FB66B01D000D00001B98304011051F1
:10068000600BE842E842E842E842E842010801E043
:100690003AD011510B0A31E0080A21E0090A19E0A9
:1006A000080A09E00B0A05E0080A01E02CD02CD862
:1006B0002AD02BD828D00001020EB06F0001BC0E4A
:1006C000B16F000EB26F0001B9930001010EB56F5A
:1006D0001AD00001020EB06F13C4BCF014D0000198
:1006E000020EB06F0001BD0EB16F000EB26F0001BF
:1006F000B9930001010EB56F06D00001020EB06F74
:1007000012C4BDF000D01200120012000001BE6B36
:100710001E0E716E0401400E096F200E0A6F040E4A
:100720000B6F880E086F0401600E0E6F040E0F6FC2
:10073000400E0C6F1200D9CFE6FFE1CFD9FFE65291
:10074000FC0EDB50400805E2400EF36EFC0EF3CFCA
:10075000DBFFDF6AFC0EDB50DF5C19E2DF50E76E87
:10076000FD0EDBCFE9FFFE0EDBCFEAFFE750E92607
:10077000000EEA22EF50E66EDF50EA6A600FE96E83
:10078000040EEA22E552E750EF6EDF2AE3D7FC0EB3
:10079000DBCF0DF4400E04010C170C7D880E0C13FA
:1007A000E552E552E7CFD9FF1200D9CFE6FFE1CFFE
:1007B000D9FF0001BE6B040108BF30D0FC0EDBCFB7
:1007C00020F00951D880205403E2FC0E09C4DBFF5D
:1007D0000001BE6BFC0EDB50BE5D19E2BE51EA6A41
:1007E000200FE96E040EEA22EF50E66EBE51E76E6E
:1007F000FD0EDBCFE9FFFE0EDBCFEAFFE750E92677
:10080000000EEA22E552E750EF6EBE2BE3D704015B
:10081000400E096F0817087D880E08130001BE51AD
:1008200000D0E552E7CFD9FF120004011051600B50
:10083000E842E842E842E842E842000901E098D094
:100840001151080A01E186D0010A72E00F0A0AE09C
:10085000030A01E08DD00001010EB06F0001040E0B
:10086000B86F86D00001010EB06F040113050AE1D4
:100870000001720EB16F090EB26F120E0001B56F5A
:10088000B66B53D0020E135D1EE11251F66EF76A7D
:10089000D890F636F7366A0EF6260A0EF7220900C9
:1008A000F5CFB1F00A00F5CFB2F0020E0001F76A01
:1008B000B125F66EB251F7220900F5CFB5F00A0066
:1008C000F5CFB6F032D0030E135D2DE1030E125DAD
:1008D00010E10001000EB16F000EB26FB1C0E9FF70
:1008E000B2C0EAFFEF500001B56FB66B0001B993DB
:1008F0003FD01251F66EF76AD890F636F7366E0E84
:10090000F6260A0EF7220900F5CFB1F00A00F5CF5E
:10091000B2F0B1C0F6FFB2C0F7FF0800F550000119
:10092000B56FB66B02D00001B06B0001B98320D067
:100930000001010EB06F12C4BAF00401125104E1BB
:100940000001050EB86F05D00001060EB86F86ECE9
:1009500003F00ED00001010EB06F0001BA0EB16FAE
:10096000000EB26F0001B9930001010EB56F00D007
:1009700012001201000200000008D8043300020037
:10098000010203020902290001010280F0090400AA
:10099000000203000000092101000001221D0007E0
:1009A0000581034000010705010340000109022001
:1009B0000001020480F00904000002FF00000007AB
:1009C00005810340000107050103400001040309FC
:1009D0000434034D006900630072006F0063006817
:1009E0000069007000200054006500630068006E1C
:1009F000006F006C006F0067007900200049006EF6
:100A00000063002E0048035000490043006B00695A
:100A10000074002000320020004D00690063007265
:100A2000006F0063006F006E00740072006F006C56
:100A3000006C00650072002000500072006F0067BB
:100A400000720061006D006D00650072000600FF1D
:100A50000901A10119012940150026FF007508951B
:100A6000408102190129409102C08409AD09CD09D4
:100A7000D109050A0806080E6D6E6DBAFED7686AC0
:100A8000110E696E0001020EB86F12006D6A696A7C
:100A90000001B86B12006850040B09E06950040BA8
:100AA00006E06D92699468A402D06894FCD76850FF
:100AB000010B04E06950010B01E023D86850200BC2
:100AC00006E06950200B03E070B07090689A030E46
:100AD0000001B85D01E214D00001BF6B040EBF5DE0
:100AE0000FE26850080B0BE06950080B08E016ECA9
:100AF00000F0000901E168960001BF2BEFD700D09C
:100B00001200686A7B0E696E6E6A160E706E68A6B9
:100B100008D06896000000000000000000000000FF
:100B2000F6D76D9898EC01F00001BA6B0001030E46
:100B3000B86F12002A0EF66E000EF76E000EF86EF9
:100B400000010900F550AA6F0900F550AB6F03E1F1
:100B5000AA6701D03DD00900F550A56F0900F550F6
:100B6000A66F0900F550A76F09000900F550E96E5E
:100B70000900F550EA6E090009000900F550A86F58
:100B80000900F550A96F09000900F6CFACF0F7CFC6
:100B9000ADF0F8CFAEF0A5C0F6FFA6C0F7FFA7C036
:100BA000F8FF0001A85302E1A95307E00900F5503E
:100BB000EE6EA807F8E2A907F9D7ACC0F6FFADC002
:100BC000F7FFAEC0F8FF0001AA07000EAB5BBFD76E
:100BD0001200D9CFE6FFE1CFD9FF030EE126938AB9
:100BE000F18E580EE66E36EC06F0E55281AA0CD076
:100BF000FE0EF66E7F0EF76EF86A0800F550DF6E97
:100C0000DF5002E000EF10F01FD83BEC05F04BEC9A
:100C100005F086EC02F0D950010FE96EDACFEAFF59
:100C2000EE50ED1001E18B70010EDB06020E01E2C9
:100C3000DB06EDD7030EE15C02E2E16AE552E16E0C
:100C4000E552E7CFD9FF1200140E6F6E0001B86BAA
:100C50000001B96B0001BA6B8B90949012003BECD1
:100C600005F06FBE02D04BEC05F01200FF0EE35012
:100C7000276EEF0E01D0F30EE76EE72E3DEF06F084
:100C80000C0E266EE76AE72E43EF06F0262E42EFA3
:100C900006F0272E3BEF06F01200000EF36E00EE7A
:100CA00000F0040E01D81200EA6002D0EE6AFCD710
:100CB000F350E9601200EE6AFCD713EE00F023EE69
:100CC00000F0F86A259C9AEC05F06BEC06F0E9EC74
:100CD00005F0FBD712001200FFFFFFFFFFFFFFFF31
:100CE000FFFFFFFFFFFFFFFFFFFFFFFFFFFFFFFF14
:100CF000FFFFFFFFFFFFFFFFFFFFFFFFFFFFFFFF04
:100D0000FFFFFFFFFFFFFFFFFFFFFFFFFFFFFFFFF3
:100D1000FFFFFFFFFFFFFFFFFFFFFFFFFFFFFFFFE3
:10200000B7EF3EF01200FFFFD1EF3AF01200FFFFF2
:10201000FFFFFFFFFFFFFFFFD1EF3AF01200FFFFCE
:10202000FFFFFFFFFFFFFFFFFFFFD9CFE6FFE1CF7D
:10203000D9FFE652030ED26EA194A08492809282C0
:102040000D0EC16E030EC06E9284809489949286A8
:102050008096899692888998899A929A8A96938688
:102060008A889398938AF18E8A9493948B90949013
:102070008B9294928B949494949C8B8C8B9E949E34
:10208000020EDF6E0001030E016F0001090E026FE8
:102090000001040E036FF00EE66E44EC2AF0E552E8
:1020A000230828E11E0EDF5C25E2DF50FE0BE8422C
:1020B000F00FE66E44EC2AF0E552E66EDF50EA6A75
:1020C000000FE96E000EEA22E552E750EF6EDF28BE
:1020D000EA6A000FE96E000EEA22EF6ADF50EA6A50
:1020E000000FE96E000EEA22EF5001E103D0020E6C
:1020F000DF26D8D7020EDF240001006F3E6A000100
:10210000E76B0001010EE86F0201030EE06F0201B0
:10211000E16B0201010EE26FB9EC19F09BEC17F0D4
:1021200093EC17F06DEC17F00001400ED880E355EA
:10213000010EE4550EE30001C00EE35D000EE4590C
:1021400008E30001E651AF0804E3500E0001E65D2C
:1021500009E20001E36B010EE46F0001E56B000191
:10216000800EE66F080ED56E040ECA6E4F0ECB6E53
:102170000C0EBD6E1D0EBE6E0001400EE06F000124
:102180003E0EE16F00013C0EE26F02017E0EFA6F1F
:1021900002012D0EFB6F070EB46EB56AF28CF28E43
:1021A000C7EC3BF0040EE66E44EC2AF0E552500812
:1021B0001CE1050EE66E44EC2AF0E5524B0815E1F1
:1021C000060EE66E44EC2AF0E55232080EE1070EE8
:1021D000E66E44EC2AF0E5523D6E7FEC36F0020EDE
:1021E0003E6E546A0201890E006FE552E552E7CF58
:1021F000D9FF120004010CBFFDD7400EE66E400E61
:10220000E66E020EE66E4CEC3AF0E552E552E5520F
:10221000B4EC3DF01200D9CFE6FFE1CFD9FF020EBA
:10222000E126DF6A010EDB6A81BA02D00001E78D88
:10223000400EE66E000EE66E020EE66E88EC3AF098
:10224000E552E552E552000803E2DE52010EDD6E72
:102250003E0406E1010EDB5002E076EC2FF012D2D4
:10226000020E3E5C09E1010EDB5004E0760E020135
:10227000005D02E011DA06D20001E8B37ADA010E5D
:10228000DB5001E1FFD1DF50EA6A000FE96E020E78
:10229000EA22EF50546E5450420A27E0340A05E017
:1022A0002C0A01E025D0DF2AE9D111EC1DF0020E45
:1022B0003E5C19E1080ED56E8A883E6AE668040E17
:1022C000E66E22EC2AF0E552E552E668050EE66E6F
:1022D00022EC2AF0E552E552E668060EE66E22ECA4
:1022E0002AF0E552E552DF2AC9D1D9EC1CF0C6D15B
:1022F000A00E545C03E2400EDF6EC0D15450B9080A
:1023000003E2400EDF6EBAD1A00E545E549E5446D6
:10231000080E5426F9505424D8B0FA2AF96E1AD06F
:102320003FD06BD06ED071D07AD091D0B1D0B4D034
:10233000BDD0C0D0C3D0C6D0C9D0CBD0CDD0D0D0E6
:1023400005D10DD115D11ED121D129D12AD131D11B
:102350007ED194D1DF28EA6A000FE96E020EEA22EC
:10236000EF50E66E020EDF24EA6A000FE96E020EFD
:10237000EA22EF50E66EE1EC15F0E552E552030E6D
:10238000DF24EA6A000FE96E020EEA22EF50E66EE1
:1023900006EC17F0E5520201FA6F040EDF26D9D7DA
:1023A000DF28EA6A000FE96E020EEA22EFCFE0F0C2
:1023B000020EDF24EA6A000FE96E020EEA22EF50F5
:1023C000E66E06EC17F0E552010F0001E16F020E18
:1023D0000001E15D0001E26F030EDF24EA6A000FF5
:1023E000E96E020EEA22EF50E66E06EC17F0E552B7
:1023F0000201FB6F040EDF26ACD7F1EC1CF0DF2AE4
:10240000A8D74EEC18F0DF2AA4D7DF2AD9CFE6FFF1
:10241000DACFE6FF53EC1AF0E552E5529AD7DF2AFD
:10242000DF28EA6A000FE96E020EEA22EF50E66E3C
:10243000DF50EA6A000FE96E020EEA22EF50E66E04
:1024400068EC19F0E552E552020EDF2682D7DF2A4A
:10245000DF50EA6A000FE96E020EEA22EF50E66EE4
:10246000DF28406A000F3F6E020E40223FC0E6FFA9
:1024700040C0E6FF1CEC1DF0E552E552E552DF508E
:10248000EA6A000FE96E020EEA22EF28DF2661D722
:102490009BEC17F0DF2A5DD7DF2AD9CFE6FFDACF32
:1024A000E6FFD4EC19F0E552E55253D793EC17F060
:1024B000DF2A4FD7C7EC18F0DF2A4BD7B9EC19F059
:1024C000DF2A47D71AEC19F0DF2A43D7400EDF6E18
:1024D00040D7FF00DF2A3DD7A3EC17F0DF2A39D71A
:1024E000DF28EA6A000FE96E020EEA22EF500001CF
:1024F000E36FE46B020EDF24EA6A000FE96E020E5E
:10250000EA22EFCF3FF0406A3FBE40683FC040F054
:102510003F6A3F500001E32740500001E423030ECF
:10252000DF24EA6A000FE96E020EEA22EFCFE5F03F
:10253000040EDF24EA6A000FE96E020EEA22EFCFF2
:10254000E6F04AEC17F0050EDF2603D7DF2AD9CFD5
:10255000E6FFDACFE6FFB3DAE552E552FAD6DF2A34
:10256000D9CFE6FFDACFE6FF2ADAE552E552F1D617
:102570008B8EDF2AD9CFE6FFDACFE6FF83D9E5528B
:10258000E552E7D6DF2ACAD98B9EE3D6DF2ADFCF12
:10259000E6FF16EC2FF0E552040EDF26DAD6DF2A2E
:1025A000D8D6DF2ADFCFE6FF2DD9E552400EDF6E09
:1025B000D0D6DF2ADF50DF2AEA6A000FE96E020E6A
:1025C000EA22EF505F6EDF50DF2AEA6A000FE96E01
:1025D000020EEA22EF50546EDF50DF2AEA6A000F43
:1025E000E96E020EEA22EF50566EDF50DF2AEA6AE9
:1025F000000FE96E020EEA22EF50586EDF50DF2A1C
:10260000EA6A000FE96E020EEA22EF50596EDF50BF
:10261000DF2AEA6A000FE96E020EEA22EF505A6ED4
:10262000DF50DF2AEA6A000FE96E020EEA22EF2885
:102630005B6EDF50DF2AEA6A000FE96E020EEA22C3
:10264000EF505E6E8B8EBEEC2DF08B9E82D6DF2A15
:10265000DF28EA6A000FE96E020EEA22EF50E66E0A
:10266000DF50EA6A000FE96E020EEA22EF50E66ED2
:1026700065D9E552E552020EDF266BD6400EDF5CCF
:1026800001E201D6020EE15C02E2E16AE552E16E8E
:10269000E552E7CFD9FF1200F29A870ED56EF2A469
:1026A00029D0D20ED76E3A0ED66EF294542A5450D8
:1026B000050801E2546A040E545C06E2010E54144B
:1026C000E8B08A88E8A08A98300E0001E71512E089
:1026D0008A8881BAFED78F0E0001E717F00EE66EEA
:1026E0008CEC3EF0E55281AAFED7F00EE66E8CEC43
:1026F0003EF0E5520001E7AD3AD08A881EEC31F099
:102700008A8881AAFED7546A300E0001E71502E0DC
:1027100081BAFED7FC0E0001E81506E0080EE66E51
:102720005EEC36F0E55210D0390406E1040EE66E98
:102730005EEC36F0E55208D03650371005E0060E54
:10274000E66E5EEC36F0E552F00EE66E8CEC3EF096
:10275000E55281AAFED7F00EE66E8CEC3EF0E55213
:102760008F0E0001E7170001E86B0001E79D8B90D9
:102770001200D9CFE6FFE1CFD9FFE6523D501AE073
:102780003D50DF6E3D6A3A50E66EB9EC27F0E552F7
:10279000DF50010805E23B50E66EB9EC27F0E55248
:1027A000DF50020805E23C50E66EB9EC27F0E55236
:1027B0003D50E6E10201E551E61108E0A050020BB0
:1027C00005E1EEEC27F0396EA182A0828150100B5A
:1027D00014E1C250020B11E10201FA51C45C0AE299
:1027E0000C0E0201FC5D03E18A948A8802D002018A
:1027F000FC2B02D00201FC6BC282E552E552E7CF0E
:10280000D9FF1200D9CFE6FFE1CFD9FFFE0EDBCF13
:10281000E6FF34EC2FF0E552000930E0020E3E6E88
:10282000546A500EE66E040EE66E22EC2AF0E55273
:10283000E5524B0EE66E050EE66E22EC2AF0E552EE
:10284000E552320EE66E060EE66E22EC2AF0E552F6
:10285000E552FE0EDB50030FEA6A000FE96E020E2E
:10286000EA22EF503D6E3D50E66E070EE66E22EC1A
:102870002AF0E552E5520201890E006FE552E7CFDA
:10288000D9FF1200D9CFE6FFE1CFD9FFF29EDCECF1
:102890003BF0050EC26EC282FD0EDBCFE9FFFE0EDD
:1028A000DBCFEAFFEF50EF2AEA6A000FE96E020E73
:1028B000EA22EF50346EFD0EDBCFE9FFFE0EDBCFD8
:1028C000EAFFEF50EF2AEA6A000FE96E020EEA22F1
:1028D000EF50356E366A376A386A396A3A6A3D6A45
:1028E0000001E88392968986928492888A94899AD4
:1028F0002E0EB46EA50EB56E0C0EE66ED3EC3EF049
:10290000E5529D90A092910ECD6E910EB16EA19C5C
:10291000A08CF28EE552E7CFD9FF1200F29E0001A3
:10292000E893A09C9D90A092CD6AB16A070EB46E08
:10293000B56A9286C7EC3BF0F28E1200D9CFE6FF63
:10294000E1CFD9FF030EE126FD0EDB50416E426A56
:1029500041C042F0416AFE0EDB50000141243F6E4F
:10296000000E4220406E010E3FC0DBFF020E40C051
:10297000DBFFDF6ADF503F6E406AD890405004E6CC
:10298000800E3F5C000E405810E2010EDBCFE9FFE5
:10299000DB2A020EDBCFEAFF01E3DB2AEF50E66E13
:1029A000B9EC27F0E552DF2AE5D7030EE15C02E23D
:1029B000E16AE552E16EE552E7CFD9FF1200D9CFC7
:1029C000E6FFE1CFD9FF050EE126FD0EDBCFE9FFE3
:1029D000FE0EDBCFEAFFEF50EF2AEA6A000FE96E46
:1029E000020EEA22040EEFCFDBFFFD0EDBCFE9FF84
:1029F000FE0EDBCFEAFFEF50EF2AEA6A000FE96E26
:102A0000020EEA22EF50E66ED950020FE96EDACFDD
:102A1000EAFFE552E750EE6EED6AD950020FE96E1B
:102A2000DACFEAFF200ED880EE54000EED5407E214
:102A3000200EF36E020EF3CFDBFF030EDB6AD950DC
:102A4000020FE96EDACFEAFFEE50ED1001E12DD072
:102A5000DE6ADD6ADECF3FF0DDCF40F0020EDBCF75
:102A600041F0030EDBCF42F041503F5C42504058F2
:102A70001AE2040EDBCFF3FFDB2AF350E66E44ECE0
:102A80002AF0E552E66EDECFE9FFDDCFEAFF400E29
:102A9000E926020EEA22E552E750EF6EDF2A010E28
:102AA00001E3DB2AD7D7FAEC10F0050EE15C02E275
:102AB000E16AE552E16EE552E7CFD9FF1200D9CFC6
:102AC000E6FFE1CFD9FF050EE126FD0EDBCFE9FFE2
:102AD000FE0EDBCFEAFFEF50EF2AEA6A000FE96E45
:102AE000020EEA22040EEFCFDBFFFD0EDBCFE9FF83
:102AF000FE0EDBCFEAFFEF50EF2AEA6A000FE96E25
:102B0000020EEA22EF50E66ED950020FE96EDACFDC
:102B1000EAFFE552E750EE6EED6AD950020FE96E1A
:102B2000DACFEAFF200ED880EE54000EED5407E213
:102B3000200EF36E020EF3CFDBFF030EDB6AD950DB
:102B4000020FE96EDACFEAFFEE50ED1001E12FD06F
:102B5000DE6ADD6ADECF3FF0DDCF40F0020EDBCF74
:102B600041F0030EDBCF42F041503F5C42504058F1
:102B70001EE2FD0EDBCFE9FFFE0EDBCFEAFFEF50DA
:102B8000EF2AEA6A000FE96E020EEA22EF50E66EC3
:102B9000040EDBCFF3FFDB2AF350E66E22EC2AF0C3
:102BA000E552E552DF2A010E01E3DB2AD3D7050EF9
:102BB000E15C02E2E16AE552E16EE552E7CFD9FF5E
:102BC0001200D9CFE6FFE1CFD9FF030EE126FE0EBA
:102BD000DB50426E436A42C043F0426AFD0EDB5056
:102BE000000142243F6E000E4320406E416A40BE09
:102BF00041683FC0DFFF010E40C0DBFF020E41C055
:102C0000DBFFD9CFE9FFDACFEAFF060EE76ED890F7
:102C1000020EEB32010EEB32EF32E706F8E1E5C0CF
:102C20003FF0406A416A3FAE02D040684168D9CF68
:102C3000E9FFDACFEAFF3F50EE264050EE22415046
:102C4000EE22E6C03FF0406A416AD9CFE9FFDACF11
:102C5000EAFF3FC02CF040C02DF041C02EF0EECF77
:102C600027F0EECF28F0EFCF29F0D9EC3CF026C0CA
:102C7000EDFF25C0EDFF24C0EFFFD9CFE9FFDACF8C
:102C8000EAFFD890020EEB32010EEB32EF32080E63
:102C9000426ED9CFE9FFDACFEAFF42501F0BEECFE9
:102CA0003FF0EECF40F0EECF41F006E0D890413259
:102CB00040323F32E806FAE13F50BE6ED9CFE9FF1D
:102CC000DACFEAFFEE52EE6AEE6ACF0EBD14426E24
:102CD000436A446A020E486ED9CFE9FFDACFEAFFB1
:102CE00048501F0BEECF45F0EECF46F0EECF47F049
:102CF00006E0D890473246324532E806FAE14250C3
:102D000045103F6E43504610406E44504710416E90
:102D10003F50BD6E030EE15C02E2E16AE552E16EF6
:102D2000E552E7CFD9FF1200D9CFE6FFE1CFD9FFB7
:102D3000040EE126FD0EDBCF3FF0FE0EDBCF40F0B0
:102D4000000E3FC0DBFF010E40C0DBFF020EDB6A5E
:102D5000030EDB6AE3C03FF0E4C040F0416A426A20
:102D6000D9CFE9FFDACFEAFF3FC02BF040C02CF00B
:102D700041C02DF042C02EF0EECF26F0EECF27F06E
:102D8000EECF28F0EFCF29F054EC3EF025C0EDFF58
:102D900024C0EDFF23C0EDFF22C0EFFFD9CFE9FF34
:102DA000DACFEAFF080EE76ED890030EEB32020E80
:102DB000EB32010EEB32EF32E706F6E1D9CFE9FF55
:102DC000DACFEAFFD880FF0EEE54FF0EEE54000E6D
:102DD000EE54000EEE5406E2DE68DE68DE6ADD6A5E
:102DE000DD52DD52DFCF3FF0010EDBCF40F03FC0C0
:102DF000F3FF40C0F4FF00D0040EE15C02E2E16AA0
:102E0000E552E16EE552E7CFD9FF1200D9CFE6FFD8
:102E1000E1CFD9FF020EE126E3C03FF0E4C040F06D
:102E2000000ED8803F56020E40563FC0DEFF40C025
:102E3000DDFFFE0EDB503F6E406AD9CFE9FFDACFEF
:102E4000EAFF3FC02DF040C02EF0EECF28F0EDCFCE
:102E500029F0BBEC3CF026C0EEFF27C0EDFFD9CF38
:102E6000E9FFDACFEAFF080E0F0B06E0EC52D8902C
:102E7000ED32EF32E806FAE1DF5000D03F6E020E8D
:102E8000E15C02E2E16AE552E16E3F50E552E7CFD4
:102E9000D9FF1200E3C0E6FFE66A22EC2AF0E55211
:102EA000E552E4C03FF0406A3F50E66E010EE66E28
:102EB00022EC2AF0E552E552E5C0E6FF020EE66E8E
:102EC00022EC2AF0E552E552E6C0E6FF030EE66E7C
:102ED00022EC2AF0E552E5521200E66A44EC2AF0B0
:102EE000E5520001E36FE46B010EE66E44EC2AF05C
:102EF000E5523F6E406A3FC040F03F6A3F500001DC
:102F0000E32740500001E423020EE66E44EC2AF071
:102F1000E5520001E56F030EE66E44EC2AF0E5523F
:102F20000001E66F12000001E96B0001EA6B00018D
:102F3000EB6BEC6B12000201E36B0201E46B02012C
:102F4000E56BE66B1200D9CFE6FFE1CFD9FF060EA5
:102F5000E126DE6ADD6A020EDB6A030EDB6A040E1E
:102F6000DB6A050EDB6A040EDB6A050EDB6A040E03
:102F7000DBCF3FF0050EDBCF40F0D890405004E6A9
:102F8000200E3F5C000E40581EE2040EDBCFE9FF2E
:102F9000050EDBCFEAFF030EEA02F3CFEAFF030ED2
:102FA000E902F3CFE9FFF450EA26800EE926020E8B
:102FB000EA22EF50DE26000EDD22040EDB2A050E8B
:102FC00001E3DB2AD4D7040EDB6A050EDB6A040EAC
:102FD000DBCF3FF0050EDBCF40F0DECF41F0DDCFA1
:102FE00042F040504218E8AE02D0423404D0415082
:102FF0003F5C425040581EE2040EDB500001F425B5
:103000000F01E96E050EDB500001F5210F01EA6E9C
:10301000EF503F6E406AD950020FE96EDACFEAFFF7
:103020003F50EE264050ED22040EDB2A050E01E350
:10303000DB2ACDD7DECF3FF0DDCF40F03F5002019D
:10304000406FDECF3FF0DDCF40F040C03FF0406A40
:103050003FC041F2FF0EE76E020EDBCF3FF0030EE2
:10306000DBCF40F0E7503F16406A3FC042F2020E0D
:10307000DBCF3FF0030EDBCF40F040C03FF0406AB3
:103080003FC043F2FAEC10F0060EE15C02E2E16AA6
:10309000E552E16EE552E7CFD9FF1200D9CFE6FF46
:1030A000E1CFD9FF020EE126DCEC3BF0040EE66E28
:1030B00060D8E552C450416E426A41C042F0416A54
:1030C000C350000141243F6E000E4220406E3FC0BD
:1030D000DEFF40C0DDFFDECFE6FFDDCFE6FF24DE12
:1030E000E552E552F3CFDEFFF4CFDDFFDFCF40F254
:1030F000DECF3FF0DDCF40F040C03FF0406A3FC040
:1031000041F2E66A36D8E552C450416E426A41C087
:1031100042F0416AC350000141243F6E000E42203C
:10312000406E3FC0DEFF40C0DDFFDECFE6FFDDCFFB
:10313000E6FFFADDE552E552F3CFDEFFF4CFDDFF27
:10314000DFCF42F2DECF3FF0DDCF40F040C03FF0B6
:10315000406A3FC043F2FAEC10F0C7EC3BF0020EBD
:10316000E15C02E2E16AE552E16EE552E7CFD9FFA8
:103170001200D9CFE6FFE1CFD9FFFE0EDB28C26EE9
:10318000C282C2B2FED7E552E7CFD9FF1200D9CF33
:10319000E6FFE1CFD9FF020EE126010EEBC0DBFF17
:1031A000010EDB503F0803E2DE523F0EDD6E010EE2
:1031B000DBCF40F2010EDF6E010EDB50D880DF5412
:1031C00023E30001EA51EA2BEA6A600FE96E000E80
:1031D000EA22EF50E66EDF50EA6A400FE96E020E17
:1031E000EA22E552E750EF6E0001EA513F6E406A75
:1031F000D890405004E6800E3F5C000E405802E339
:103200000001EA6BDF2AD8D7010EDB503F6E406A1F
:103210003F500001EB5F40500001EC5BFAEC10F016
:10322000020EE15C02E2E16AE552E16EE552E7CFAF
:10323000D9FF1200D9CFE6FFE1CFD9FF020EE12678
:10324000010EEBC0DBFF010EDB50400803E2DE5253
:10325000400EDD6EDF6A010EDB50DF5C23E2000111
:10326000EA51EA2BEA6A600FE96E000EEA22EF509B
:10327000E66EDF50EA6A400FE96E020EEA22E5527E
:10328000E750EF6E0001EA513F6E406AD89040501F
:1032900004E6800E3F5C000E405802E30001EA6B3A
:1032A000DF2AD9D7010EDB503F6E406A3F50000144
:1032B000EB5F40500001EC5BFAEC10F0020EE15CB9
:1032C00002E2E16AE552E16EE552E7CFD9FF120072
:1032D000D9CFE6FFE1CFD9FF200EF36EFE0EDBCF94
:1032E000F4FFF350F45C0DE2FE0EDB50030DF3CF60
:1032F000E9FFF4CFEAFF800EE926020EEA22EF5042
:1033000003E10001E88B31D0FE0EDB50030DF3CF5B
:10331000E9FFF4CFEAFF800EE926020EEA22EF5021
:10332000E66EFE0EDB50030DF3CFE9FFF4CFEAFFAC
:10333000800EE926020EEA22EE5200010001F4514D
:10334000EE243F6E00010001F551EE20406E3FC0BB
:10335000E6FF40C0E6FF70DBE552E552E552FD0EA8
:10336000DB06FD0EDB500008CFE3E552E7CFD9FFC7
:103370001200D9CFE6FFE1CFD9FFE652DF6A200E77
:10338000DF5C0DE2DF50030DF3CFE9FFF4CFEAFF7E
:10339000800EE926020EEA22EF6ADF2AF0D7E55214
:1033A000E552E7CFD9FF1200D9CFE6FFE1CFD9FF31
:1033B000040EE126FD0EDBCFE9FFFE0EDBCFEAFFB8
:1033C000EF50EF2AEA6A000FE96E020EEA22EF5090
:1033D000E66ED950020FE96EDACFEAFFE552E75008
:1033E000EE6EED6A020EDB500201E52500013F6E34
:1033F000030EDB500201E6210001406E000ED88072
:103400003F54010E405403E20001E88F42D0DE6ACF
:10341000DD6ADECF3FF0DDCF40F0020EDBCF41F0C2
:10342000030EDBCF42F041503F5C4250405831E246
:10343000FD0EDBCFE9FFFE0EDBCFEAFFEF50EF2AF8
:10344000EA6A000FE96E020EEA22EF50E66E020110
:10345000E351E32BEA6A000FE96E010EEA22E5521E
:10346000E750EF6E0201E3513F6E406AD890405042
:1034700004E6000E3F5C010E405802E30201E36BDC
:103480000201E52B000EE623DF2A010E01E3DB2A11
:10349000C0D7040EE15C02E2E16AE552E16EE5525A
:1034A000E7CFD9FF1200D9CFE6FFE1CFD9FF080E51
:1034B000E126FD0EDBCFE9FFFE0EDBCFEAFFEF28B2
:1034C000EA6A000FE96E020EEA22EFCF3FF0406A8F
:1034D0003FBE4068040E3FC0DBFF050E40C0DBFF6F
:1034E000040EDBCF3FF0050EDBCF40F0403404E2AA
:1034F0003F503D08000E405403E20001E88D4FD2DA
:10350000FD0EDBCFE9FFFE0EDBCFEAFFEF50EA6AEC
:10351000000FE96E020EEA22EFCF3FF0406A3FBE95
:103520004068060E3FC0DBFF070E40C0DBFF020E07
:10353000DB6A030EDB6ADE6ADD6ADECF3FF0DDCFD9
:1035400040F0D890405004E6200E3F5C000E4058FA
:1035500023E2DECFE9FFDDCFEAFF030EEA02F3CF7D
:10356000EAFF030EE902F3CFE9FFF450EA26800EEA
:10357000E926020EEA22EF503F6E406AD950020F50
:10358000E96EDACFEAFF3F50EE264050ED22DF2A07
:10359000010E01E3DB2AD1D7060EDBCFE9FF070ED0
:1035A000DBCFEAFF030EEA02F3CFEAFF030EE902E4
:1035B000F3CFE9FFF450EA26800EE926020EEA2254
:1035C000EF503F6E406AD950020FE96EDACFEAFF42
:1035D0003F50EE5E4050ED5A040EDBCF3FF0050E3B
:1035E000DBCF40F0020EDBCF41F0030EDBCF42F029
:1035F000000ED8804156030E425642504018E8AEA5
:1036000002D0403404D03F50415C4050425803E265
:103610000001E88DC4D1060EDBCF3FF0070EDBCFF3
:1036200040F0403404E23F501F08000E405403E2D3
:103630000001E88DB4D1060EDBCFE9FF070EDBCF2A
:10364000EAFF030EEA02F3CFEAFF030EE902F3CF2B
:10365000E9FFF450EA26800EE926020EEA22EF5036
:1036600001E106D1060EDBCFE9FF070EDBCFEAFF53
:10367000030EEA02F3CFEAFF030EE902F3CFE9FFFC
:10368000F450EA26800EE926020EEA22EF503F6E41
:10369000406A000ED8803F56030E40563F06000E8B
:1036A000405A040E3FC0DBFF050E40C0DBFF060E94
:1036B000DBCFE9FF070EDBCFEAFF030EEA02F3CF11
:1036C000EAFF030EE902F3CFE9FFF450EA26800E89
:1036D000E926020EEA22EE52EECFDEFFEDCFDDFF4D
:1036E000DECF3FF0DDCF40F0040EDBCF41F0050E22
:1036F000DBCF42F040504218E8AE02D0423404D052
:1037000041503F5C4250405835E2060EDBCFE9FFA6
:10371000070EDBCFEAFF030EEA02F3CFEAFF030E48
:10372000E902F3CFE9FFF450EA26800EE926020E03
:10373000EA22EF500001406AF4253F6EF551402225
:10374000DE503F24E96EDD504020EA6EEF50E66E19
:10375000DE500001F4250F01E96EDD500001F52176
:103760000F01EA6EE552E750EF6EDF2A010E01E32A
:10377000DB2AB6D7DE6ADD6ADECF3FF0DDCF40F070
:10378000D890405004E6200E3F5C000E405870E296
:10379000DECFE9FFDDCFEAFF030EEA02F3CFEAFF57
:1037A000030EE902F3CFE9FFF450EA26800EE92682
:1037B000020EEA22EECF3FF0EECF40F0EFCF41F025
:1037C000060EDBCFE9FF070EDBCFEAFF030EEA02AE
:1037D000F3CFEAFF030EE902F3CFE9FFF450EA2644
:1037E000800EE926020EEA22EE52EECF42F0EFCF33
:1037F00043F0000143504118E8AE02D0413404D0F8
:103800004050425C415043582EE2060EDBCFE9FFA8
:10381000070EDBCFEAFF030EEA02F3CFEAFF030E47
:10382000E902F3CFE9FFF450EA26800EE926020E02
:10383000EA22EF503F6E406ADECFE9FFDDCFEAFFBC
:10384000030EEA02F3CFEAFF030EE902F3CFE9FF2A
:10385000F450EA26800EE926020EEA22EE523F508C
:10386000EE5E4050ED5ADF2A010E01E3DB2A84D7D9
:10387000FD0EDBCFE9FFFE0EDBCFEAFFEF28EA6AA1
:10388000000FE96E020EEA22EF50E66E060EDBCF65
:10389000E9FF070EDBCFEAFF030EEA02F3CFEAFFF0
:1038A000030EE902F3CFE9FFF450EA26800EE92681
:1038B000020EEA22E552E750EF6E060EDBCFE9FF7B
:1038C000070EDBCFEAFF030EEA02F3CFEAFF030E97
:1038D000E902F3CFE9FFF450EA26800EE926020E52
:1038E000EA22EE52020EDBCFEEFF030EDBCFEDFF3E
:1038F000020E3F6EFD0EDBCFE9FFFE0EDBCFEAFFCF
:103900003F50EF26DE6ADD6ADECF3FF0DDCF40F0CC
:10391000060EDBCFE9FF070EDBCFEAFF030EEA025C
:10392000F3CFEAFF030EE902F3CFE9FFF450EA26F2
:10393000800EE926020EEA22EF50000140AE02D0CE
:10394000D89003D03F5C000E405829E2FD0EDBCF3B
:10395000E9FFFE0EDBCFEAFFEF50EF2AEA6A000F25
:10396000E96E020EEA22EF50E66E020EDB50000115
:10397000F42500013F6E030EDB500001F52100012C
:10398000406EDE503F24E96EDD504020EA6EE55285
:10399000E750EF6EDF2A010E01E3DB2AB5D7080EF0
:1039A000E15C02E2E16AE552E16EE552E7CFD9FF60
:1039B0001200F29EAFEC3DF0840EA66EFE0EF66E87
:1039C0007F0EF76EF86AF56A0C00550EA76EAA0E08
:1039D000A76EA6824E0EE66E8CEC3EF0E552FF001E
:1039E0001200F00E0001E71781A402D00001E78762
:1039F00080AA02D00001E78581B802D00001E783E8
:103A000081A602D00001E781E7C040F2E8C041F2A0
:103A10008F0E0001E7170001E86B8B90FAEC10F0B5
:103A200012000201020E406F0201200E416F0201DE
:103A3000426BFAEC10F01200D9CFE6FFE1CFD9FFCC
:103A40000D0EE126DF6A0B0EDB6A0C0EDB6AF29AC2
:103A5000070ED56EFC0EDB5004E0FC0EDB503D087B
:103A600004E20001E88B6DEF24F0FE0E0001E81582
:103A700002E06DEF24F0FC0EDB50DF5C02E36DEF43
:103A800024F0DF50E76EFD0EDBCFE9FFFE0EDBCF4B
:103A9000EAFFE750E926000EEA22EF50546EB30E1B
:103AA000545C04E2FC0EDB50DF6EDFD7D50E545CB5
:103AB00001E2D3D3D50E545E549E5446080E5426CC
:103AC000F9505424D8B0FA2AF96EAED3A3D3E8D271
:103AD00009D358D324D3E1D2D9D26FD266D251D2EE
:103AE00048D2EFD121D2E9D1D4D19BD163D13CD1FD
:103AF0004ED1F7D0E6D0D2D0BAD0A2D079D072D001
:103B000067D05CD045D02FD02CD029D026D023D060
:103B10001FD01BD017D013D011D00FD00CD000D095
:103B2000DCEC3BF08A98E80EE66E8CEC3EF0E55259
:103B3000C7EC3BF090D38A888ED38DD38CD38B8EF9
:103B40008A8489D38B9E8A9486D30C0EBA6E83D3D3
:103B5000BA6A8B9280D3898A7ED3899A7CD38B80F0
:103B60007AD38B9078D3DF2ADF50E76EFD0EDBCF60
:103B7000E9FFFE0EDBCFEAFFE750E926000EEA225E
:103B8000EFCFE0F2E0C2E6FF8EEC28F0E55263D31F
:103B9000DF2A080EE66EDF50E76EFD0EDBCFE9FF91
:103BA000FE0EDBCFEAFFE750E926000EEA22EF50D7
:103BB000E66E1EEC28F0E552E5524DD3080EE66E97
:103BC000EEEC27F0E66E1EEC28F0E552E55243D30A
:103BD000080EE66E70EC27F0E552E66EB9EC27F0C1
:103BE000E55239D3080EE66E70EC27F0E55233D378
:103BF000DF2ADF50E76EFD0EDBCFE9FFFE0EDBCFE5
:103C0000EAFFE750E926000EEA22EF50E66EDF50A9
:103C1000E76EFD0EDBCFE9FFFE0EDBCFEAFFE750DC
:103C2000E926000EEA22010EE926000EEA22EF50F4
:103C3000E66E1EEC28F0E552E552020EDF260CD3AC
:103C4000DF2ADF50E76EFD0EDBCFE9FFFE0EDBCF94
:103C5000EAFFE750E926000EEA22EF50E66EEEECAE
:103C600027F0E66E1EEC28F0E552E552F4D2DF2A8A
:103C7000DF50E76EFD0EDBCFE9FFFE0EDBCFEAFF84
:103C8000E750E926000EEA22EF50E66E70EC27F0CE
:103C9000E552E66EB9EC27F0E552DDD2DF2ADF50BF
:103CA000E76EFD0EDBCFE9FFFE0EDBCFEAFFE7504C
:103CB000E926000EEA22EF50E66E70EC27F0E5529E
:103CC000CAD2DF2ADF50E76EFD0EDBCFE9FFFE0E22
:103CD000DBCFEAFFE750E926000EEA22EFCFE1F260
:103CE000BAD20B0EDB500EE0040EDB06040EDB50E6
:103CF00005E10B0EDB6A030EDF26AED2050EDB50AC
:103D0000DF6EAAD2010EF36E0B0EF3CFDBFFDF5096
:103D1000E76EFD0EDBCFE9FFFE0EDBCFEAFFE750DB
:103D2000E926000EEA22010EE926000EEA22EF50F3
:103D3000DF5CE76E050EE7CFDBFFDF50E76EFD0EC1
:103D4000DBCFE9FFFE0EDBCFEAFFE750E926000EEE
:103D5000EA22020EE926000EEA22040EEFCFDBFF74
:103D6000050EDB50DF6E78D2DF2ADF50E76EFD0EE6
:103D7000DBCFE9FFFE0EDBCFEAFFE750E926000EBE
:103D8000EA22EF50E66E08EC27F0E55264D2DF2A13
:103D9000DF50E76EFD0EDBCFE9FFFE0EDBCFEAFF63
:103DA000E750E926000EEA22EF50E66E9CEC24F084
:103DB000E55251D20001E905EA6A600FE96E000E92
:103DC000EA22010EEFCFDBFFDF50E76EFD0EDBCF07
:103DD000E9FFFE0EDBCFEAFFE750E926000EEA22FC
:103DE000010EE926000EEA22EF50F36E010EDB50C1
:103DF000F35C14E1DF50E76EFD0EDBCFE9FFFE0E52
:103E0000DBCFEAFFE750E926000EEA22020EE926A0
:103E1000000EEA22EF50DF24DF6E02D0030EDF2611
:103E20001BD20001E905EA6A600FE96E000EEA2282
:103E3000010EEFCFDBFF010EDBCF3FF0DF50E76E6F
:103E4000FD0EDBCFE9FFFE0EDBCFEAFFE750E926F0
:103E5000000EEA22010EE926000EEA22EF50D88079
:103E60003F5414E2DF50E76EFD0EDBCFE9FFFE0E9C
:103E7000DBCFEAFFE750E926000EEA22020EE92630
:103E8000000EEA22EF50DF24DF6E02D0030EDF26A1
:103E9000E3D1DF50E76EFD0EDBCFE9FFFE0EDBCF97
:103EA000EAFFE750E926000EEA22010EE926000E9D
:103EB000EA22EF50DF24DF6ECFD1FC0EDB50DF6E45
:103EC000CBD1DF2ADF50DF2AE76EFD0EDBCFE9FF23
:103ED000FE0EDBCFEAFFE750E926000EEA22EF50A4
:103EE000406A000F3F6E0F0E4022090E3FC0DBFFFD
:103EF0000A0E40C0DBFFDF50DF2AE76EFD0EDBCF8E
:103F0000E9FFFE0EDBCFEAFFE750E926000EEA22CA
:103F1000EF50E66E090EDBCFE9FF0A0EDBCFEAFFBA
:103F2000E552E750EF6E98D1DF2ADF50E76EFD0EC5
:103F3000DBCFE9FFFE0EDBCFEAFFE750E926000EFC
:103F4000EA22EF50406A000F3F6E0F0E4022090E2A
:103F50003FC0DBFF0A0E40C0DBFF090EDBCFE9FFED
:103F60000A0EDBCFEAFFEF50E66EB9EC27F0E55220
:103F700072D1DF2A2DEC25F0E66EB9EC27F0E55280
:103F80006BD1DF2ADF50DF2AE76EFD0EDBCFE9FFC2
:103F9000FE0EDBCFEAFFE750E926000EEA22EF50E3
:103FA000E66EAFEC24F0E55257D1DF2AEEEC27F0B5
:103FB000E66EAFEC24F0E5524FD10C0EDB5016E06C
:103FC000070EDB06080E01E2DB06D950070FE96E8B
:103FD000DACFEAFFEE50ED1005E10C0EDB6A020EBF
:103FE000DF263AD1060EDB50DF6E36D1DF50E76EAA
:103FF000FD0EDBCFE9FFFE0EDBCFEAFFE750E9263F
:10400000000EEA22010EE926000EEA22EF50DF5CE4
:10401000E76E060EE7CFDBFFEEEC27F0E66ED95039
:10402000070FE96EDACFEAFFE552E750EE6EED6A70
:10403000EEEC27F0416E426A286A010E296E41C0FB
:104040002DF042C02EF08EEC3CF026C03FF027C091
:1040500040F0D950070FE96EDACFEAFF3F50EE2665
:104060004050ED22D950070FE96EDACFEAFFEE504B
:10407000ED1003E1020EDF26EFD0010EF36E0C0E01
:10408000F3CFDBFF060EDB50DF6EE6D0AEEC28F0A0
:10409000E66EB9EC27F0E552DED0EEEC27F0DBD08F
:1040A000040EE66E010EE66E1EEC28F0E552E552B7
:1040B000080EE66EE66A1EEC28F0E552E552080EA0
:1040C000E66E27EC27F0E552E66EB9EC27F0E552F4
:1040D000080EE66E27EC27F0E552E66EB9EC27F005
:1040E000E552B9D0040EE66EE66A1EEC28F0E55201
:1040F000E552080EE66EE66A1EEC28F0E552E5523F
:10410000080EE66EE66A1EEC28F0E552E552080E4F
:10411000E66EE66A1EEC28F0E552E5529CD0DF2AF6
:10412000040EE66EE66A1EEC28F0E552E552080E33
:10413000E66EDF50DF2AE76EFD0EDBCFE9FFFE0EF5
:10414000DBCFEAFFE750E926000EEA22EF50E66EE9
:104150001EEC28F0E552E552080EE66EDF50DF2A2D
:10416000E76EFD0EDBCFE9FFFE0EDBCFEAFFE75087
:10417000E926000EEA22EF50E66E1EEC28F0E5522A
:10418000E5526AD0DF2A040EE66EE66A1EEC28F0DD
:10419000E552E552080EE66EDF50DF2AE76EFD0EAF
:1041A000DBCFE9FFFE0EDBCFEAFFE750E926000E8A
:1041B000EA22EF50E66E1EEC28F0E552E552080EBA
:1041C000E66EDF50DF2AE76EFD0EDBCFE9FFFE0E65
:1041D000DBCFEAFFE750E926000EEA22EF50E66E59
:1041E0001EEC28F0E552E552080EE66EDF50DF2A9D
:1041F000E76EFD0EDBCFE9FFFE0EDBCFEAFFE750F7
:10420000E926000EEA22EF50E66E1EEC28F0E55299
:10421000E55222D0080EE66E27EC27F0E552E66E56
:10422000B9EC27F0E55217D0DF2ADF50E76EFD0E1C
:10423000DBCFE9FFFE0EDBCFEAFFE750E926000EF9
:10424000EA22EF50E66E27EC27F0E552E66EB9EC75
:1042500027F0E55200D0DF2A08D4B30E545E549EF6
:104260005446080E5426F9505424D8B0FA2AF96E50
:104270006AD270D227D3C6D216D3C7D273D250D245
:104280003CD213D2D7D1ACD185D17ED16AD163D102
:1042900057D13FD135D12DD119D10ED104D1FCD078
:1042A000E8D0E4D0E0D0D8D0C2D0AAD081D06ED0AF
:1042B00001D035D0DF2A040EE66EE66A1EEC28F047
:1042C000E552E552040EE66EDF50E76EFD0EDBCFE1
:1042D000E9FFFE0EDBCFEAFFE750E926000EEA22F7
:1042E000EF50E66E1EEC28F0E552E552080EE66E41
:1042F000EEEC27F0E66E1EEC28F0E552E552080ED3
:10430000E66EE66A1EEC28F0E552E552040EE66E13
:10431000020EE66E1EEC28F0E552E5529CD7DF2A2D
:10432000040EE66EE66A1EEC28F0E552E552040E35
:10433000E66EDF50E76EFD0EDBCFE9FFFE0EDBCF52
:10434000EAFFE750E926000EEA22EF50E66E1EEC87
:1043500028F0E552E552080EE66EEEEC27F0E66E28
:104360001EEC28F0E552E552080EE66EEEEC27F062
:10437000E66E1EEC28F0E552E552040EE66E020EE3
:10438000E66E1EEC28F0E552E55265D7DF2ADF50D5
:10439000E76EFD0EDBCFE9FFFE0EDBCFEAFFE75055
:1043A000E926000EEA22EF50E66EA1DAE55253D775
:1043B000DF2ADF50E76EFD0EDBCFE9FFFE0EDBCF1D
:1043C000EAFFE750E926000EEA22EF50E66EDF50E2
:1043D000E76EFD0EDBCFE9FFFE0EDBCFEAFFE75015
:1043E000E926000EEA22010EE926000EEA22EF502D
:1043F000E66E56EC28F0E552E552020EDF262CD789
:10440000DF2ADF50E76EFD0EDBCFE9FFFE0EDBCFCC
:10441000EAFFE750E926000EEA22EF50E66EEEECE6
:1044200027F0E66E56EC28F0E552E55214D7DF2A65
:10443000DF50E76EFD0EDBCFE9FFFE0EDBCFEAFFBC
:10444000E750E926000EEA22EFCFE2F2E2C2E6FFF1
:10445000C1EC28F0E552FFD6D5EC28F0E66EB9ECB9
:1044600027F0E552F8D6E6EC28F0F5D6FCEC28F07B
:10447000F2D6DF2ADF50E76EFD0EDBCFE9FFFE0E3E
:10448000DBCFEAFFE750E926000EEA22EF50E66EA6
:1044900012EC29F0E552DFD6EEEC27F0E66E12ECD6
:1044A00029F0E552D8D6E66A7BEC29F0E552E66EB3
:1044B000B9EC27F0E552CFD60F0EE66E7BEC29F073
:1044C000E552E66EB9EC27F0E552C5D6DF2ADF509B
:1044D000E76EFD0EDBCFE9FFFE0EDBCFEAFFE75014
:1044E000E926000EEA22EF50E66EE2EC29F0E552F2
:1044F000B2D6EEEC27F0E66EE2EC29F0E552ABD650
:10450000E66AE2EC29F0E552E66EB9EC27F0E552F6
:10451000A2D6DF2ADF50E76EFD0EDBCFE9FFFE0EED
:10452000DBCFEAFFE750E926000EEA22EF50E66E05
:10453000E2EC29F0E552E66EB9EC27F0E5528BD6B5
:10454000EEEC27F0E66EE2EC29F0E552E66EB9EC0F
:1045500027F0E55280D67ADBE66EB9EC27F0E5521B
:104560007AD6DF2ADF50DF2AE76EFD0EDBCFE9FFC8
:10457000FE0EDBCFEAFFE750E926000EEA22EF50FD
:10458000E66EDCDAE55268D6EEEC27F0E66ED6DAB7
:10459000E55261D6CEDB020EF3CFDBFF030EF4CF84
:1045A000DBFFFF0EE76E020EDBCF3FF0030EDBCF2B
:1045B00040F0E7503F16406A3F50E66EB9EC27F0F6
:1045C000E552020EDBCF3FF0030EDBCF40F040C0E0
:1045D0003FF0406A3F50E66EB9EC27F0E5523BD61B
:1045E000DF2AE66ADF50E76EFD0EDBCFE9FFFE0E45
:1045F000DBCFEAFFE750E926000EEA22010EE926AA
:10460000000EEA22EF50E66EDF50E76EFD0EDBCFC4
:10461000E9FFFE0EDBCFEAFFE750E926000EEA22B3
:10462000EF50E66E53EC2AF0E552E552E552020EE9
:10463000DF2612D6DF2ADF50E76EFD0EDBCFE9FF63
:10464000FE0EDBCFEAFFE750E926000EEA22020E5B
:10465000E926000EEA22EF50E66EDF50E76EFD0E0F
:10466000DBCFE9FFFE0EDBCFEAFFE750E926000EC5
:10467000EA22010EE926000EEA22EF50E66EDF5034
:10468000E76EFD0EDBCFE9FFFE0EDBCFEAFFE75062
:10469000E926000EEA22EF50E66E53EC2AF0E552CE
:1046A000E552E552030EDF26D7D5DF2ADF50E76E4D
:1046B000FD0EDBCFE9FFFE0EDBCFEAFFE750E92678
:1046C000000EEA22010EE926000EEA22EF50E66E05
:1046D000DF50E76EFD0EDBCFE9FFFE0EDBCFEAFF1A
:1046E000E750E926000EEA22EF50E66EA8EC2BF028
:1046F000E552E552020EDF26AFD5DF2ADF50E76E26
:10470000FD0EDBCFE9FFFE0EDBCFEAFFE750E92627
:10471000000EEA22EF50E66EECEC2BF0E5529BD552
:10472000DF2ADF50E76EFD0EDBCFE9FFFE0EDBCFA9
:10473000EAFFE750E926000EEA22EF50E66E0DECA4
:104740002CF0E55288D5E66AE66A70EC2DF0E55269
:10475000E55281D5010EE66EE66A70EC2DF0E55269
:10476000E55279D5DF2A010EE66EDF50E76EFD0EC9
:10477000DBCFE9FFFE0EDBCFEAFFE750E926000EB4
:10478000EA22EF50E66EDF50E76EFD0EDBCFE9FF69
:10479000FE0EDBCFEAFFE750E926000EEA22010E0B
:1047A000E926000EEA22EF50E66EDF50E76EFD0EBE
:1047B000DBCFE9FFFE0EDBCFEAFFE750E926000E74
:1047C000EA22020EE926000EEA22EF50E66EDF50E2
:1047D000E76EFD0EDBCFE9FFFE0EDBCFEAFFE75011
:1047E000E926000EEA22030EE926000EEA22EF5027
:1047F000E66E3DEC2CF03F6E050EE15E3F50040E80
:10480000DF262AD51FEC2DF026D5DF2ADF50E76EF4
:10481000FD0EDBCFE9FFFE0EDBCFEAFFE750E92616
:10482000000EEA22EF50E66EDF50E76EFD0EDBCFA2
:10483000E9FFFE0EDBCFEAFFE750E926000EEA2291
:10484000010EE926000EEA22EF50E66EDF50E76E19
:10485000FD0EDBCFE9FFFE0EDBCFEAFFE750E926D6
:10486000000EEA22020EE926000EEA22EF50E66E62
:10487000DF50E76EFD0EDBCFE9FFFE0EDBCFEAFF78
:10488000E750E926000EEA22030EE926000EEA228E
:10489000EF50E66ECEEC2CF0E552E552E552E552D3
:1048A000040EDF26D9D49ADBE66E98DBE66E96DB43
:1048B000E66E94DBE66ECEEC2CF0E552E552E55266
:1048C000E552C9D4010EE66E010EE66E70EC2DF0D5
:1048D000E552E552C0D435EF1DF00D0EE15C02E269
:1048E000E16AE552E16EE552E7CFD9FF1200D9CF78
:1048F000E6FFE1CFD9FF0201E351E32BEA6A000FA3
:10490000E96E010EEA22FE0EDBCFEFFF0201E3515A
:104910003F6E406AD890405004E6000E3F5C010EA6
:10492000405802E30201E36B0201E52B000EE6238F
:10493000E552E7CFD9FF1200D9CFE6FFE1CFD9FF8B
:10494000F294FE0EDB50FF0DF350D76ED66AD58E73
:10495000F2A4FED7D59EE552E7CFD9FF1200D9CFFA
:10496000E6FFE1CFD9FFF29ECD90A40ED76E730E75
:10497000D66EF294D58E8050080B04E1F250040BF1
:1049800001E1F9D7F2B45DD089949294600EE66E9D
:10499000C5EC3EF0E55289848050080B04E0F250EB
:1049A000040B01E1F9D7F2B44CD0FE0EDB50546E8B
:1049B000F2B646D080A6FCD7899454BE898480B6CE
:1049C000FED7F2B63DD080A6FCD7899454BC89842A
:1049D00080B6FED7F2B634D080A6FCD7899454BAFC
:1049E000898480B6FED7F2B62BD080A6FCD78994F6
:1049F00054B8898480B6FED7F2B622D080A6FCD700
:104A0000899454B6898480B6FED7F2B619D080A6B0
:104A1000FCD7899454B4898480B6FED7F2B610D0FE
:104A200080A6FCD7899454B2898480B6FED7F2B6AA
:104A300007D080A6FCD7899454B0898480B6FED76D
:104A40000000F2A402D00001E885D59EF28ECD8050
:104A500000D0E552E7CFD9FF1200CD90F29EA40E10
:104A6000D76E730ED66EF294D58E8050080B04E18B
:104A7000F250040B01E1F9D7F2B454D08994929426
:104A8000600EE66EC5EC3EF0E55289848050080B5E
:104A900004E0F250040B01E1F9D79284F2B442D061
:104AA000546AF2B63ED080A6FCD780B6FED780B45A
:104AB000548EF2B636D080A6FCD780B6FED780B42E
:104AC000548CF2B62ED080A6FCD780B6FED780B428
:104AD000548AF2B626D080A6FCD780B6FED780B422
:104AE0005488F2B61ED080A6FCD780B6FED780B41C
:104AF0005486F2B616D080A6FCD780B6FED780B416
:104B00005484F2B60ED080A6FCD780B6FED780B40F
:104B10005482F2B606D080A6FCD780B6FED780B409
:104B20005480000089849294F2A402D00001E885A8
:104B3000D59EF28ECD80545000D01200D9CFE6FF22
:104B4000E1CFD9FFF29ECD90A40ED76E730ED66E34
:104B5000F294D58E92848050040B04E0F250040B42
:104B600001E1F9D7F2B45FD092968986600EE66EC5
:104B7000C5EC3EF0E55289968050040B04E1F250FA
:104B8000040B01E1F9D792869294F2B44CD0FE0E58
:104B9000DB50546EF2B646D080A6FCD7899454BE42
:104BA000898480B6FED7F2B63DD080A6FCD7899422
:104BB00054BC898480B6FED7F2B634D080A6FCD728
:104BC000899454BA898480B6FED7F2B62BD080A6D9
:104BD000FCD7899454B8898480B6FED7F2B622D027
:104BE00080A6FCD7899454B6898480B6FED7F2B6E5
:104BF00019D080A6FCD7899454B4898480B6FED796
:104C0000F2B610D080A6FCD7899454B2898480B6BD
:104C1000FED7F2B607D080A6FCD7899454B0898419
:104C200080B6FED70000F2A402D00001E885600E35
:104C3000E66EC5EC3EF0E552D59EF28ECD809284B4
:104C4000929600D0E552E7CFD9FF1200CD90F29EA8
:104C5000A40ED76E730ED66EF294D58E92848050C9
:104C6000040B04E0F250040B01E1F9D7F2B455D083
:104C700092968986600EE66EC5EC3EF0E552899606
:104C80008050040B04E1F250040B01E1F9D7928447
:104C90009286F2B442D0546AF2B63ED080A6FCD7D7
:104CA00080B6FED780B4548EF2B636D080A6FCD73C
:104CB00080B6FED780B4548CF2B62ED080A6FCD736
:104CC00080B6FED780B4548AF2B626D080A6FCD730
:104CD00080B6FED780B45488F2B61ED080A6FCD72A
:104CE00080B6FED780B45486F2B616D080A6FCD724
:104CF00080B6FED780B45484F2B60ED080A6FCD71E
:104D000080B6FED780B45482F2B606D080A6FCD717
:104D100080B6FED780B454800000F2A402D0000117
:104D2000E885D59E92849296F28ECD80545000D024
:104D30001200D9CFE6FFE1CFD9FF030EE126DF6AEB
:104D40008B8EF294800ED76ED66AD58EF2AE02D0DC
:104D5000010EDF6EF29E80A40AD0F2A407D0D59E89
:104D6000DF0401E1F28EF36AF46A48D0F4D780B42C
:104D70000AD0F2A407D0D59EDF0401E1F28EF36AD7
:104D8000F46A3CD0F4D7800ED76ED66AF29480A431
:104D90000AD0F2A407D0D59EDF0401E1F28EF368B9
:104DA000F4682CD0F4D7D59EDF0401E1F28ED65002
:104DB000E66ED950010FE96EDACFEAFFE552E7500F
:104DC000EE6EED6A7F0ED7143F6E406A3FC040F032
:104DD0003F6AD950010FE96EDACFEAFF3F50EE2665
:104DE0004050ED228B9E010EDBCF3FF0020EDBCF59
:104DF00040F03FC0F3FF40C0F4FF00D0030EE15C81
:104E000002E2E16AE552E16EE552E7CFD9FF120016
:104E1000D9CFE6FFE1CFD9FFF294D768080EE66E4E
:104E2000D3EC3EF0E552FE0EDB0402E10CD002D0E2
:104E3000FE0EDB06FE0EDB50FF0DF350D66ED58E58
:104E4000F2A4FED7D59EE552E7CFD9FF1200D9CF05
:104E5000E6FFE1CFD9FFE6529284546AFE0EDB50A2
:104E6000556E020E0201E15D0CE280B45480898629
:104E7000000000000000899600005442552EF5D72E
:104E800018D00201E105566E565080B454808986D0
:104E900000000000000000000000E82EFBD789960B
:104EA0005650000000000000E82EFBD75442552E5B
:104EB000EBD7FE0EDBCFE6FF080EE552D880E754B5
:104EC000070B04E05442549EE806FCE10201E0A313
:104ED0009294545000D0E552E552E7CFD9FF12002A
:104EE000D9CFE6FFE1CFD9FFE6529284546AFE0E95
:104EF000DB50556E020E0201E15D0CE28986000076
:104F00000000000080B45480899600005442552E61
:104F1000F5D718D00201E105566E89860000000021
:104F20005650000000000000E82EFBD780B45480EB
:104F300089965650000000000000E82EFBD754422E
:104F4000552EEBD7FE0EDBCFE6FF080EE552D880DC
:104F5000E754070B04E05442549EE806FCE10201CA
:104F6000E0A39294545000D0E552E552E7CFD9FF28
:104F70001200D9CFE6FFE1CFD9FF010E0001406A50
:104F8000EB253F6EEC514022800ED8803F54000E3E
:104F9000405403E20001E8871DD00001E951E92BEC
:104FA000EA6A600FE96E000EEA22FE0EDBCFEFFF29
:104FB0000001E9513F6E406AD890405004E6800EEF
:104FC0003F5C000E405802E30001E96B0001EB2B4F
:104FD000000EEC23E552E7CFD9FF1200D9CFE6FF50
:104FE000E1CFD9FFE6520201E551E61104E10001EB
:104FF000E889000E1ED00201E451E42BEA6A000F9A
:10500000E96E010EEA22EFCFDFFF0201E507000E95
:10501000E65B0201E4513F6E406AD890405004E6DE
:10502000000E3F5C010E405802E30201E46BDF50CA
:1050300000D0E552E552E7CFD9FF1200D9CFE6FF05
:10504000E1CFD9FFE652FE0EDB50546EFD0EDB5071
:10505000556E020E0201E15D0CE254A0899454B039
:10506000898400008986000089965442552EF5D720
:1050700018D00201E105566E54A0899454B0898479
:105080005650000000000000E82EFBD789865650DD
:10509000000000000000E82EFBD789965442552EF0
:1050A000EBD7E552E552E7CFD9FF1200D9CFE6FFA3
:1050B000E1CFD9FFE652FE0EDB50546EFD0EDB5001
:1050C000556E020E0201E15D0CE254A0899454B0C9
:1050D000898489860000899600005442552EF5D7B0
:1050E00018D00201E105566E54A0899454B0898409
:1050F00056508986000000000000E82EFBD78996F4
:105100005650000000000000E82EFBD75442552EF8
:10511000EBD7E552E552E7CFD9FF1200D9CFE6FF32
:10512000E1CFD9FFFE0EDBA402D0898601D089969B
:10513000FE0EDBA602D0898401D08994FE0EDBA08E
:1051400002D0928601D09296FE0EDBA202D092840B
:1051500001D09294E552E7CFD9FF1200D9CFE6FFF4
:10516000E1CFD9FFE652DF6A80B4DF8280A602D0A9
:10517000000EDB80DF5000D0E552E552E7CFD9FFCB
:105180001200D9CFE6FFE1CFD9FFFE0EDBA202D09D
:10519000898801D08998FE0EDBA002D0928801D0C8
:1051A0009298E552E7CFD9FF1200D9CFE6FFE1CFC1
:1051B000D9FFE652DF6A80A802D0000EDB80DF5004
:1051C00000D0E552E552E7CFD9FF12008B8E8986D9
:1051D000060EE66ED3EC3EF0E55289989298060EE4
:1051E000E66ED3EC3EF0E5528996060EE66ED3EC01
:1051F0003EF0E552928812008996060EE66ED3ECD8
:105200003EF0E55289989298060EE66ED3EC3EF099
:10521000E5528986060EE66ED3EC3EF0E5529288A2
:105220008B9E1200D9CFE6FFE1CFD9FFFE0EDB50F7
:10523000546E080E556E8998020E0201E15D23E25C
:1052400054AE929854BE928800D000D000D0898687
:10525000000000D000D000D000D08996000000D01F
:1052600000D05446552EECD7928800D000D000D004
:1052700000D000D08986000000D000D000D080B8D7
:10528000558089962FD00201E151E824FF0F566E18
:1052900054AE929854BE92885650000000D000D070
:1052A00000D0E82EFAD78986565000D000D000D022
:1052B000E82EFDD7899600005446552EE9D79288EE
:1052C000565000D000D0000000D000D000D0E82E12
:1052D000FAD78986565000D000D0E82EFDD780B886
:1052E000558089965550000802E20001E885E55294
:1052F000E7CFD9FF1200D9CFE6FFE1CFD9FF546A3B
:10530000080E556E010E566E9288020E0201E15D86
:1053100014E2544600D000D000D000D000008986AE
:1053200000D000D000D0000080B85480899600D012
:1053300000D000D0552EEDD725D00201E151E82450
:10534000FF0F566E5446000000D0565000D000D0DB
:1053500000D00000E82EFAD78986565000D000D041
:10536000E82EFDD780B85480899600D0552EEAD714
:105370000000565000D000D000D000D000D0000077
:10538000E82EFAD78998FE0EDB5001E1929856502C
:1053900000D000D000D000D000D00000E82EFAD716
:1053A0008986565000D000D0E82EFDD700D08996CF
:1053B00000D0000000009288545000D0E552E7CFA2
:1053C000D9FF1200D9CFE6FFE1CFD9FFE6528B8E8D
:1053D000FE0EDB50546E080E556E020E0201E15DAA
:1053E0000DE254AE899854BE8988898654465490FB
:1053F00080B454808996552EF4D71BD00201E10564
:10540000566E54AE899854BE8988565000000000EC
:105410000000E82EFBD789865446549080B454800F
:105420005650000000000000E82EFBD78996552E4C
:10543000E8D789988B9E545000D0E552E552E7CFCB
:10544000D9FF1200D9CFE6FFE1CFD9FFE652DF6ADC
:10545000FE0EDB50A96EFD0EDB50A86EA66AA68478
:10546000F2AE02D0010EDF6EF29E550EA76EAA0EAE
:10547000A76EA682DF0401E1F28EA6B2FED7E55246
:10548000E552E7CFD9FF1200D9CFE6FFE1CFD9FF30
:10549000FE0EDB50A96EA66AA680A85000D0E55289
:1054A000E7CFD9FF1200D9CFE6FFE1CFD9FF040E35
:1054B000E126DF6A010EDB6A0201E151010808E220
:1054C000120E566E0F0EF36E030EF3CFDBFF07D0F6
:1054D000C60E566E030EF36E030EF3CFDBFF898804
:1054E0009298180EE66ED3EC3EF0E552020E3F6E37
:1054F000FD0EDBCFE7FF3F50E726FD0EE7CFDBFFDA
:10550000480ED56E550E546E8998D66AF294D58E93
:10551000F2AE02D0010EDF6EF29EFD0EDB06020E31
:10552000DB6A020EDBCF3FF0080EE76E3F18E8AEF5
:1055300002D0E73402D0E7503F5C21E28950EF0B04
:1055400054AE1009F2A4FED7896E5650D626929812
:10555000F294549E54468950556EFD0EDB5005E181
:10556000FC0EDB5002E1558801D05598F2A4FED71D
:1055700089785650D626F294020EDB2AD2D755509F
:10558000F2A4FED7896E5650D626F294010EDB5057
:1055900007E0FD0EDB50000803E220DD546E03D06F
:1055A000FE0EDB50546EF2A4FED789785650D626F4
:1055B000F294F2A4FED792885650D626F294030EA7
:1055C000DBCFE6FFD3EC3EF0E552010EDB5009E005
:1055D0008050100B06E00001E885FD0EDB6AFC0E32
:1055E000DB6AF2A4FED700005650D626F294030ED2
:1055F000DBCFE6FFD3EC3EF0E552010EDB5009E0D5
:105600008050100B06E10001E885FD0EDB6AFC0E00
:10561000DB6ADE52010EDD6EFD0EDB50000801E29A
:105620007CD7FC0EDBCFF3FFDB06F350000801E371
:105630007FD0546A020EDB6A020EDBCF3FF0080E09
:10564000E76E3F18E8AE02D0E73402D0E7503F5C87
:1056500030E2F2A4FED70000D66AF2948950556E6B
:10566000FC0EDB5002E1558801D05598030EDB0497
:10567000E66ED3EC3EF0E55280B807D0F2B402D02B
:1056800080A8FCD75650D66E06D0F2B402D080B8AF
:10569000FCD75650D66EF294030EDBCFE6FFD3EC68
:1056A0003EF0E552549E544680B8542A020EDB2A3E
:1056B000C3D75550F2A4FED7896E5650D62692987D
:1056C000F2945450E66E55DCE552F2A4FED7897888
:1056D0005650D626F294F2A4FED792885650D6267B
:1056E000F294030EDBCFE6FFD3EC3EF0E552010E61
:1056F000DB5007E08050100B04E00001E885FC0E51
:10570000DB6AF2A4FED700005650D626F294030EB0
:10571000DBCFE6FFD3EC3EF0E552010EDB5007E0B5
:105720008050100B04E10001E885FC0EDB6A79D79C
:10573000DF0401E1F28E070ED56E9288040EE15C63
:1057400002E2E16AE552E16EE552E7CFD9FF1200CD
:10575000D9CFE6FFE1CFD9FFE652FE0EDB5001E1E3
:105760000FD0546AFD0EDB50556EDF6AFE0EDB5023
:10577000DF5C06E270EC38F055905542DF2AF6D730
:10578000E552E552E7CFD9FF1200D9CFE6FFE1CFCE
:10579000D9FFE652FE0EDB5002E1000E18D0FD0EDE
:1057A000DB50546EFC0EDB50556E566ADF6AFE0EFF
:1057B000DB50DF5C0AE25690564270EC38F05490B1
:1057C000544255905542DF2AF2D7565000D0E55248
:1057D000E552E7CFD9FF1200D9CFE6FFE1CFD9FFDD
:1057E000030EE66E040EE66EB3DFE552E552100ED0
:1057F000E66EFE0EDBCFE6FF050EE66EC6DFE55277
:10580000E552E552010EE66E020EE66EA1DFE552AC
:10581000E552E552E7CFD9FF1200D9CFE6FFE1CF3D
:10582000D9FFE652DF6A010EE66E030EE66E90DFE8
:10583000E552E55256AE02D0010EDF6E800EE66EE6
:10584000FE0EDBCFE6FF080EE66E9FDFE552E55267
:10585000E5525650E824DF12DFCFE6FFB9EC27F01F
:10586000E552010EE66E020EE66E72DFE552E5527B
:10587000E552E552E7CFD9FF1200D9CFE6FFE1CFDD
:10588000D9FF020EE126DF6A010EDB6A010EE66E29
:10589000030EE66E5DDFE552E55256AE02D0010E14
:1058A000DF6EE66AFB0EDBCFE6FF080EE66E6DDF0D
:1058B000E552E552E5525650E824DF12FA0EDB506D
:1058C00005E0DFCFE6FFB9EC27F0E552DF6A56AE20
:1058D00002D0010EDF6EE66AFC0EDBCFE6FF080E9B
:1058E000E66E53DFE552E552E5525650E824DF12EA
:1058F000FA0EDB5005E0DFCFE6FFB9EC27F0E5520A
:10590000DF6A56AE02D0010EDF6EE66AFD0EDBCF17
:10591000E6FF080EE66E39DFE552E552E5525650D5
:10592000E824DF12FA0EDB5005E0DFCFE6FFB9EC2A
:1059300027F0E552010EDFCFDBFFDF6A56AE02D063
:10594000010EDF6E800EE66EFE0EDBCFE6FF080E68
:10595000E66E1BDFE552E552E5525650E824DF12B1
:10596000FA0EDB5005E0DFCFE6FFB9EC27F0E55299
:10597000010EE66E020EE66EEBDEE552E552010E1A
:10598000DB5000D03F6E020EE15C02E2E16AE552BC
:10599000E16E3F50E552E7CFD9FF1200D9CFE6FFC5
:1059A000E1CFD9FF010EE66E030EE66ED1DEE552C1
:1059B000E55256BE0AD01F0EE66E050EE66EC8DE34
:1059C000E552E5520001E88536D0E66A010EE66E42
:1059D000BFDEE552E552E66AFB0EDBCFE6FF080EBE
:1059E000E66ED3DEE552E552E552E66AFC0EDBCF09
:1059F000E6FF080EE66EC9DEE552E552E552E66ABC
:105A0000FD0EDBCFE6FF080EE66EBFDEE552E55287
:105A1000E552800EE66EFE0EDBCFE6FF080EE66E68
:105A2000B4DEE552E552E552010EE66E020EE66E78
:105A30008FDEE552E552E552E7CFD9FF1200D9CF0C
:105A4000E6FFE1CFD9FFE652D76AD66AF294D58E47
:105A50000A0EE66EC1DEE552E66AE66AD00EE66E32
:105A6000040EE66EE66A09DF3F6E050EE15E3F500A
:105A7000DF6E040EDF1403E1F250040BEDE0F2A43C
:105A800004D00001E885D59E26D0090EE66EA4DE7E
:105A9000E552E66AEEEC27F0E66EEEEC27F0E66EF5
:105AA000EEEC27F0E66EEEEC27F0E66EE6DE3F6EFB
:105AB000050EE15E3F500A0EE66E8EDEE552E66AA6
:105AC000E66AC00EE66EE66AE66AD7DE3F6E050E4F
:105AD000E15E3F50D59EE552E552E7CFD9FF120077
:105AE000D9CFE6FFE1CFD9FFE652D76AD66AF29462
:105AF000D58E0A0EE66E70DEE552E66AE66AD00ED4
:105B0000E66E040EE66EE66AB8DE3F6E050EE15EF6
:105B10003F50DF6E040EDF1403E1F250040BEDE0A2
:105B2000F2A404D00001E885D59E23D0090EE66ECC
:105B300053DEE552FE0EDBCFE6FFE66AE66AE66A72
:105B4000E66A9BDE3F6E050EE15E3F50FD0EDB50C8
:105B50000FE00A0EE66E40DEE552E66AE66AC00E27
:105B6000E66EE66AE66A89DE3F6E050EE15E3F504C
:105B7000D59EE552E552E7CFD9FF1200D9CFE6FF17
:105B8000E1CFD9FF020EE126F29EDCEC3BF09284DD
:105B900092869288B9EC19F08B80E950DF6E010E85
:105BA000EACFDBFF5F5002E05F6A02D058505F6EC1
:105BB00088EC38F05E50000803E210EC39F007D0B2
:105BC0005F5003E0D5EC38F002D09AEC38F0DF50AB
:105BD000E96E010EDB50EA6E8B90C7EC3BF0F28E63
:105BE00054C040F255C041F2FAEC10F0020EE15CF4
:105BF00002E2E16AE552E16EE552E7CFD9FF120019
:105C00000100BE7D0000F400000002000000D9CFBA
:105C1000E6FFE1CFD9FFE6520401B06B0401B16B9E
:105C2000B26B396AC56AC76A280EC66E1F0EC86E87
:105C3000C584C5B4FED7E552E552E7CFD9FF1200BF
:105C4000D9CFE6FFE1CFD9FFE6528B9C67D804019C
:105C5000B06B9E960401B051B02BEA6AC00FE96E9A
:105C6000040EEA22EF50C96E9EA6FED7C5BCC584BD
:105C7000400E0401B05DEDE3C584C5B4FED7060E49
:105C8000E66E8CEC3EF0E5520401B06B0401B12BE2
:105C9000000EB2238B8CE552E552E7CFD9FF1200FC
:105CA000D9CFE6FFE1CFD9FFE65238D80109DF6E40
:105CB000C582C5B2FED79E96DF50C96E9EA6FED79E
:105CC000C5BCC5840401B06B9E96C5869EA6FED752
:105CD0000401B051B02BEA6AC00FE96E040EEA224B
:105CE000C9CFEFFF400E0401B05D02E1C58A01D0CB
:105CF000C59AC588C5B8FED7400E0401B05DE4E37F
:105D0000C584C5B4FED70401B06B0401B12B000EED
:105D1000B223E552E552E7CFD9FF1200D9CFE6FF13
:105D2000E1CFD9FF020EE126DE52A00EDD6E3D501E
:105D300007E10401B251040B02E0010EDB820CD03A
:105D40000401B251080B02E0010EDB820401B251E2
:105D5000040B02E0010EDB86C580C5B0FED79E961F
:105D6000010EDB50C96EB1C43FF0B2C440F0D89010
:105D700040323F32D89040323F323F50DF6E9EA6D5
:105D8000FED7C5BCC5849E96DF50C96EB1C43FF036
:105D9000B2C440F0060ED8903F364036E804FBE12E
:105DA0003F50DF6E9EA6FED7C5BCC5849E96DF50D1
:105DB000C96E9EA6FED7C5BCC584010EDB5000D0BF
:105DC0003F6E020EE15C02E2E16AE552E16E3F5095
:105DD000E552E7CFD9FF1200D9CFE6FFE1CFD9FFD7
:105DE0000401B051B02BEA6AC00FE96E040EEA223A
:105DF000FE0EDBCFEFFF0401B0513F0801E220DFD0
:105E0000E552E7CFD9FF12000401B0513F0803E289
:105E100047DF0401B06B0401B051B02BEA6AC00F38
:105E2000E96E040EEA22EF5000D01200D9CFE6FF4F
:105E3000E1CFD9FF3E6AFE0EDBCFE6FF15D8E55273
:105E400000090EE0FE0EDB50030FEA6A000FE96E58
:105E5000020EEA22EF503D6E010E3E6ED8DE8B80C0
:105E6000E552E7CFD9FF1200D9CFE6FFE1CFD9FF46
:105E7000FE0EDBCFF3FFDB2AF350EA6A000FE96E78
:105E8000020EEA22EF50500802E0000E20D0FE0E73
:105E9000DBCFF3FFDB2AF350EA6A000FE96E020E54
:105EA000EA22EF504B0802E0000E11D0FE0EDBCFCD
:105EB000F3FFDB2AF350EA6A000FE96E020EEA22D2
:105EC000EF50320802E0000E02D0010E00D0E55281
:105ED000E7CFD9FF1200AD0EE66E7EDFE55204017A
:105EE000B0510008F8E33E6A8B901200D9CFE6FF6C
:105EF000E1CFD9FF020EE126DF6A010EDB6ADF5037
:105F0000EA6A000FE96E020EEA22EF50840A01E10C
:105F10004ED1210A01E129D1270A01E126D1010A46
:105F200001E123D1040A01E120D1070A01E11DD1D9
:105F3000010A01E11AD1230A01E115D1010A01E1A7
:105F400012D10D0A01E10FD1010A01E10CD1080AB9
:105F500001E1FDD00E0A01E1FAD0030A01E1F7D018
:105F6000010A01E1F4D0070A01E1F1D0290A01E1B7
:105F7000EED0030A01E1EBD02E0A01E1BCD00E0AFB
:105F800001E18DD0020A54E0140A4FE0100A20E02B
:105F9000010A1EE0130A19E0030A0CE0070A06E0F2
:105FA0001B0A01E03CD1400EDF6E3AD1400EDF6E9D
:105FB00092DF36D1020EDF26DF50EA6A000FE96E6B
:105FC000020EEA22EF28DF262BD1030EDF2628D18E
:105FD000DF50DF2AEA6A000FE96E020EEA22EF5074
:105FE000E66EFADEE552DF50DF2AEA6A000FE96E5C
:105FF000020EEA22EF50E66EEFDEE552DF50DF2AB6
:10600000EA6A000FE96E020EEA22EF50E66EE4DE65
:10601000E552DF50DF2AEA6A000FE96E020EEA223B
:10602000EF50E66ED9DEE552FBD0050EDF26F8D044
:10603000DF50DF2AEA6A000FE96E020EEA22EF5013
:10604000E66ECADEE552DF50DF2AEA6A000FE96E2B
:10605000020EEA22EF50E66EBFDEE552DF50DF2A85
:10606000EA6A000FE96E020EEA22010EEFCFDBFFB3
:10607000010EDBCFE6FFB0DEE552DF50DF2AEA6A31
:10608000000FE96E020EEA22EF50E66EA5DEE55241
:10609000010EDB06010EDB500008EFE3C1D0DF503C
:1060A000DF2AEA6A000FE96E020EEA22EF50E66E7E
:1060B00093DEE552DF50DF2AEA6A000FE96E020E36
:1060C000EA22010EEFCFDBFF010EDBCFE6FF84DE1D
:1060D000E552DF50DF2AEA6A000FE96E020EEA227B
:1060E000EF50E66E79DEE552010EDB06010EDB5065
:1060F0000008EFE395D0DF50DF2AEA6A000FE96E6F
:10610000020EEA22EF50E66E67DEE552DF50DF2A2C
:10611000EA6A000FE96E020EEA22010EEFCFDBFF02
:10612000010EDBCFE6FF58DEE552DF50DF2AEA6AD8
:10613000000FE96E020EEA22EF50E66E4DDEE552E8
:10614000010EDB06010EDB500008EFE369D0DF50E3
:10615000DF2AEA6A000FE96E020EEA22EF50E66ECD
:106160003BDEE5525DD0DF2A5BD0DF50DF2AEA6AF2
:10617000000FE96E020EEA22EF50E66E2DDEE552C8
:10618000DF50DF2AEA6A000FE96E020EEA22EF50C2
:10619000E66E22DEE552DF50DF2AEA6A000FE96E82
:1061A000020EEA22EF50E66E17DEE55239D0DF50DC
:1061B000DF2AEA6A000FE96E020EEA22EF50E66E6D
:1061C0000BDEE552DF50DF2AEA6A000FE96E020EAD
:1061D000EA22EF50E66E00DEE552DF50DF2AEA6A7F
:1061E000000FE96E020EEA22EF50E66EF5DDE55291
:1061F000DF50DF2AEA6A000FE96E020EEA22EF5052
:10620000E66EEADDE552DF50DF2AEA6A000FE96E4A
:10621000020EEA22EF50E66EDFDDE55201D0DF2A02
:10622000400EDF5C01E26BD6020EE15C02E2E16A45
:10623000E552E16EE552E7CFD9FF1200D9CFE6FF74
:10624000E1CFD9FF020EE126E2DC0401400EB06F7F
:10625000DBDDDF6EDF50AB0A01E1D1D0070A01E1DF
:10626000CCD0060A01E1C9D0030A01E1C3D0010A7A
:1062700001E1BDD00F0A01E1B7D0010A01E19CD0D4
:10628000030A01E18AD0010A01E185D0050A6BE029
:10629000010A53E0FA0A50E0DC0A4CE0030A48E045
:1062A000010A36E0070A2BE0040A25E0050A21E08E
:1062B000030A11E0010A01E0A5D0A6DDE76E010E98
:1062C000E7CFDBFFA1DDE66E010EDBCFE6FF60D995
:1062D000E552E55299D098DDE76E010EE7CFDBFF7E
:1062E00093DDE66E010EDBCFE6FFB0D9E552E55255
:1062F0008BD0366A376A88DD386E86DD85D0361CED
:10630000366E371C376E80DD361A7EDD371A7CD04C
:106310007BDD586E79DD596E77DD5A6E75DD5B6E0B
:1063200081D8000904E1010E396EAD0EDF6E6CD02C
:1063300003D96AD021D968D067D066DDE76E010E37
:10634000E7CFDBFF010EDBCFE6FF5EDDE66EE1ECC3
:1063500015F0E552E55258DDE66E06EC17F0E55211
:106360000201FA6F51D050DD0001E06F4DDDE66EA5
:1063700006EC17F0E552010F0001E16F020E00017B
:10638000E15D0001E26F40DDE66E06EC17F0E552DC
:106390000201FB6F39D0B6D937D036DDE76E010E7A
:1063A000E7CFDBFF31DDE66E010EDBCFE6FF68EC09
:1063B00019F0E552E55228D027DDE76E010EE7CF50
:1063C000DBFF010EDBCFE6FFDAEC35F0E552010E24
:1063D000DBCFE6FF000EE66E020EE66E1CEC1DF053
:1063E000E552E552E55210D09BEC17F00DD0F7ECDA
:1063F00035F00AD093EC17F007D04ED805D0B9ECA1
:1064000019F002D0AD0EDF6EAD0EDF5C01E020D7DB
:10641000020EE15C02E2E16AE552E16EE552E7CF8D
:10642000D9FF120093EC17F0010EE66EE66A68ECF5
:1064300019F0E552E552010EE66E020EE66E68ECCA
:1064400019F0E552E552010EE66E010EE66E68ECBB
:1064500019F0E552E5520001EA51EA2BEA6A600FB1
:10646000E96E000EEA22EF5058160001EA51EA2BBD
:10647000EA6A600FE96E000EEA22EF50591693ECBB
:1064800017F05A50585C05E15B50595C02E1010E6F
:1064900002D0000E00D01200D9CFE6FFE1CFD9FF25
:1064A000040EE126360EDE6E000EDD6E020EDB6A95
:1064B000020EDBCF3FF00001EB513F5C000EEC55CC
:1064C0002FE20001EA51EA2BEA6A600FE96E000E42
:1064D000EA22030EEFCFDBFF385013E0020EDBA001
:1064E0000ED038A003D0030EDB9E08D0030EDB9243
:1064F000DB94DB96DB98DB9ADB9CDB9E02D0030E01
:10650000DB90030EDB503F6E406ADECFE9FFDDCF4C
:10651000EAFF3F50EE264050ED22020EDB2AC8D79C
:1065200093EC17F0040EE15C02E2E16AE552E16EE1
:10653000E552E7CFD9FF120093EC17F0010EE66E9B
:10654000E66A68EC19F0E552E552010EE66E0D0EB2
:10655000E66E68EC19F0E552E552010EE66E010EAA
:10656000E66E68EC19F0E552E552600E0001611527
:106570003A6E93EC17F012003A5001010113010E2C
:10658000E66E0F0EE66E68EC19F0E552E552120069
:10659000D9CFE6FFE1CFD9FF9BEC17F093EC17F0D2
:1065A0000201E351E32BEA6A000FE96E010EEA22D1
:1065B000FE0EDBCFEFFF0201E351E32BEA6A000F8F
:1065C000E96E010EEA22FD0EDBCFEFFF0201E3517F
:1065D000E32BEA6A000FE96E010EEA22EF6A030E6E
:1065E0000201E527000E0201E623010EE66EE66ACF
:1065F00068EC19F0E552E552010EE66E140EE66EF7
:1066000068EC19F0E552E552010EE66E010EE66EF9
:1066100068EC19F0E552E5520001EA51EA2BEA6A0A
:10662000600FE96E000EEA22EF50346E0001EA516D
:10663000EA2BEA6A600FE96E000EEA22EF50356E2F
:1066400093EC17F0E552E7CFD9FF1200D9CFE6FF60
:10665000E1CFD9FF9BEC17F093EC17F00201E35167
:10666000E32BEA6A000FE96E010EEA22FE0EDBCF91
:10667000EFFF0201E351E32BEA6A000FE96E010E1E
:10668000EA22FD0EDBCFEFFF0201E351E32BEA6AC2
:10669000000FE96E010EEA22EF6A0201E351E32BDB
:1066A000EA6A000FE96E010EEA2234C0EFFF020130
:1066B000E351E32BEA6A000FE96E010EEA2235C0CE
:1066C000EFFF050E0201E527000E0201E623010E91
:1066D000E66EE66A68EC19F0E552E552010EE66EE8
:1066E000150EE66E68EC19F0E552E552010EE66E05
:1066F000010EE66E68EC19F0E552E552E552E7CF7F
:10670000D9FF1200D9CFE6FFE1CFD9FF0A0EE1266B
:1067100004EC2FF0E66ED950060FE96EDACFEAFFEF
:10672000E552E750EE6EED6A04EC2FF0E66ED950BC
:10673000040FE96EDACFEAFFE552E750EE6EED6A3C
:10674000040EDBCF28F0050EDBCF29F0080E28C0A1
:10675000DBFF090E29C0DBFF040EDBCF3FF0050E87
:10676000DBCF40F0403404E23F503D08000E40547F
:1067700003E20001E88D14D2020EDB6A030EDB6A2D
:10678000DE6ADD6ADECF3FF0DDCF40F0D8904050CA
:1067900004E6200E3F5C000E405823E2DECFE9FF06
:1067A000DDCFEAFF030EEA02F3CFEAFF030EE902B0
:1067B000F3CFE9FFF450EA26800EE926020EEA2222
:1067C000EF503F6E406AD950020FE96EDACFEAFF10
:1067D0003F50EE264050ED22DF2A010E01E3DB2A76
:1067E000D1D7060EDBCFE9FF070EDBCFEAFF030EA2
:1067F000EA02F3CFEAFF030EE902F3CFE9FFF45018
:10680000EA26800EE926020EEA22EF503F6E406A29
:10681000D950020FE96EDACFEAFF3F50EE5E4050EA
:10682000ED5A040EDBCF3FF0050EDBCF40F0020E39
:10683000DBCF41F0030EDBCF42F0000ED880415693
:10684000030E425642504018E8AE02D0403404D005
:106850003F50415C4050425803E20001E88DA0D116
:10686000060EDBCF3FF0070EDBCF40F0403404E2F2
:106870003F501F08000E405403E20001E88D90D104
:10688000060EDBCFE9FF070EDBCFEAFF030EEA02BD
:10689000F3CFEAFF030EE902F3CFE9FFF450EA2653
:1068A000800EE926020EEA22EF5001E106D1060E23
:1068B000DBCFE9FF070EDBCFEAFF030EEA02F3CFDF
:1068C000EAFF030EE902F3CFE9FFF450EA26800E57
:1068D000E926020EEA22EF503F6E406A000ED88091
:1068E0003F56030E40563F06000E405A040E3FC06E
:1068F000DBFF050E40C0DBFF060EDBCFE9FF070E16
:10690000DBCFEAFF030EEA02F3CFEAFF030EE90250
:10691000F3CFE9FFF450EA26800EE926020EEA22C0
:10692000EE52EECFDEFFEDCFDDFFDECF3FF0DDCF6D
:1069300040F0040EDBCF41F0050EDBCF42F04050BB
:106940004218E8AE02D0423404D041503F5C42507D
:10695000405835E2060EDBCFE9FF070EDBCFEAFF3A
:10696000030EEA02F3CFEAFF030EE902F3CFE9FFD9
:10697000F450EA26800EE926020EEA22EF500001CA
:10698000406AF4253F6EF5514022DE503F24E96E07
:10699000DD504020EA6EEF50E66EDE500001F42537
:1069A0000F01E96EDD500001F5210F01EA6EE5529D
:1069B000E750EF6EDF2A010E01E3DB2AB6D7DE6A6D
:1069C000DD6ADECF3FF0DDCF40F0D890405004E6E6
:1069D000200E3F5C000E405870E2DECFE9FFDDCFB5
:1069E000EAFF030EEA02F3CFEAFF030EE902F3CF58
:1069F000E9FFF450EA26800EE926020EEA22EECFE5
:106A00003FF0EECF40F0EFCF41F0060EDBCFE9FFD5
:106A1000070EDBCFEAFF030EEA02F3CFEAFF030E15
:106A2000E902F3CFE9FFF450EA26800EE926020ED0
:106A3000EA22EE52EECF42F0EFCF43F00001435096
:106A40004118E8AE02D0413404D04050425C41507D
:106A500043582EE2060EDBCFE9FF070EDBCFEAFF3D
:106A6000030EEA02F3CFEAFF030EE902F3CFE9FFD8
:106A7000F450EA26800EE926020EEA22EF503F6E1D
:106A8000406ADECFE9FFDDCFEAFF030EEA02F3CF73
:106A9000EAFF030EE902F3CFE9FFF450EA26800E85
:106AA000E926020EEA22EE523F50EE5E4050ED5AC9
:106AB000DF2A010E01E3DB2A84D7060EDBCFE9FFD4
:106AC000070EDBCFEAFF030EEA02F3CFEAFF030E65
:106AD000E902F3CFE9FFF450EA26800EE926020E20
:106AE000EA22080EDBCFEFFF060EDBCFE9FF070E31
:106AF000DBCFEAFF030EEA02F3CFEAFF030EE9025F
:106B0000F3CFE9FFF450EA26800EE926020EEA22CE
:106B1000EE52020EDBCFEEFF030EDBCFEDFFDE6A9F
:106B2000DD6ADECF3FF0DDCF40F0060EDBCFE9FFC0
:106B3000070EDBCFEAFF030EEA02F3CFEAFF030EF4
:106B4000E902F3CFE9FFF450EA26800EE926020EAF
:106B5000EA22EF50000140AE02D0D89003D03F5C53
:106B6000000E40581DE204EC2FF0E66E020EDB50E2
:106B70000001F42500013F6E030EDB500001F521FA
:106B80000001406EDE503F24E96EDD504020EA6E89
:106B9000E552E750EF6EDF2A010E01E3DB2AC1D791
:106BA0000A0EE15C02E2E16AE552E16EE552E7CFEE
:106BB000D9FF1200D9CFE6FFE1CFD9FFE652DF6A55
:106BC000FE0EDB50DF5C0EE204EC2FF0E66EDF50D1
:106BD000EA6A000FE96E020EEA22E552E750EF6E14
:106BE000DF2AEED7E552E552E7CFD9FF1200D9CF21
:106BF000E6FFE1CFD9FF040EE12604EC2FF0E66EAC
:106C0000D950020FE96EDACFEAFFE552E750EE6E97
:106C1000ED6A020EDB500201E52500013F6E030E16
:106C2000DB500201E6210001406E000ED8803F5487
:106C3000010E405403E20001E88F36D0DE6ADD6ABF
:106C4000DECF3FF0DDCF40F0020EDBCF41F0030E90
:106C5000DBCF42F041503F5C4250405825E204EC0B
:106C60002FF0E66E0201E351E32BEA6A000FE96EB2
:106C7000010EEA22E552E750EF6E0201E3513F6E4A
:106C8000406AD890405004E6000E3F5C010E405828
:106C900002E30201E36B0201E52B000EE623DF2A8B
:106CA000010E01E3DB2ACCD7040EE15C02E2E16ACB
:106CB000E552E16EE552E7CFD9FF1200D9CFE6FFEA
:106CC000E1CFD9FFE652DF6A81AA14D0FE0EDB5075
:106CD000D880DF5408E3DF50DF2A010BE8B08B8057
:106CE000E8A08B9001D0DF6AF00EE66E8CEC3EF0EF
:106CF000E552EAD7E552E552E7CFD9FF1200D9CFE6
:106D0000E6FFE1CFD9FF020EE12607EC2EF00401E9
:106D1000400EB06F04EC2FF0E76E010EE7CFDBFF03
:106D2000010EDB50A00815E104EC2FF0DF6EDFCF81
:106D3000E6FF04EC2FF0E66EE1EC15F0E552E552CB
:106D400004EC2FF0E66E06EC17F0E5520201FA6F44
:106D500006D0010EDB50AD0801E101D0DBD7020EF9
:106D6000E15C02E2E16AE552E16EE552E7CFD9FF6C
:106D700012006C500CE16896040100513C0BE84293
:106D8000E8420D0802E10ED801D04BD808D0040E1D
:106D90006C5C03E1689657D802D0000E02D0010E59
:106DA00000D01200D9CFE6FFE1CFD9FFE6520401AF
:106DB00004AF02D00401046B0201F96B0201F16B14
:106DC0000201F26B0201F76BF86BE2EC3BF0DF6A59
:106DD000DF503F6E406A010E3F5C000E40581BE2E0
:106DE0000201F25101E017D0F76ADF34FE0BF736EB
:106DF000F66E460EF6267B0EF7220900F5CF3FF021
:106E00000800F5CF40F004D040C0FAFF3F50F96EC3
:106E1000FBDFDF2ADDD705D9E552E552E7CFD9FF01
:106E20001200020E0201F15D0CE1B9D8040100BDAF
:106E300004D00401C80E006F03D00401880E006F57
:106E400001D03ED91200040E0001ED5D0CE112C428
:106E50006EFF6E50000804E20001050EED6F03D0D6
:106E60000001030EED6F0201F10514E115D8020EC9
:106E70000201F95D04E10401840E046F0AD00401EB
:106E800004BD04D00401C80E046F03D00401880EB1
:106E9000046F01D015D91200D9CFE6FFE1CFD9FF99
:106EA000020EE1260201080EF75D000EF85912E20B
:106EB000F7C2DEFFF8C2DDFF0201F95104E1020171
:106EC000010EF96F06D00201F90503E10201020E7D
:106ED000F96F03D0080EDE6EDD6A0401049304012D
:106EE0000491010EDB5004010413DFCF05F4000E02
:106EF000DB500201F75F010EDB500201F85B02017B
:106F0000180EF56F040EF66F0001EEA320D0D9CF56
:106F1000E9FFDACFEAFFEE50ED1018E0F3C2F6FF1A
:106F2000F4C2F7FF0800F550F5C2E9FFF6C2EAFF28
:106F3000EF6E0201F52B000EF6230201F32B000E7B
:106F4000F423DF06010E01E2DB06E1D71ED0D9CF24
:106F5000E9FFDACFEAFFEE50ED1017E0F3C2E9FFE8
:106F6000F4C2EAFFEF50F5C2E9FFF6C2EAFFEF6EA6
:106F70000201F52B000EF6230201F32B000EF42381
:106F8000DF06010E01E2DB06E2D7020EE15C02E25F
:106F9000E16AE552E16EE552E7CFD9FF1200D9CFA1
:106FA000E6FFE1CFD9FF020EE126030E0401001532
:106FB000E76E010EE7CFDBFF01C4DFFFDE50020109
:106FC000F727DD500201F8230201180EF36F040EBB
:106FD000F46FD9CFE9FFDACFEAFFEE50ED1017E0FA
:106FE000F3C2E9FFF4C2EAFFEF50F5C2E9FFF6C2CF
:106FF000EAFFEF6E0201F52B000EF6230201F32BE0
:10700000000EF423DF06010E01E2DB06E2D7020EDA
:10701000E15C02E2E16AE552E16EE552E7CFD9FFB9
:1070200012006D980201F2510FE10401080E016F88
:107030000401100E026F040E036F0401840E006F32
:107040000401840E046F3BD0040110AF25D002016F
:10705000F7510401165D0201F8510401175904E2C9
:1070600016C4F7F217C4F8F217DF0201010EF16F30
:107070000401080E016F0401100E026F040E036F6D
:107080000401800E006F0401180E066F040E076FD6
:107090000401C80E046F13D00201020EF16F040147
:1070A000056B0401C80E046F0401080E016F040192
:1070B000180E026F040E036F0401C80E006F120059
:1070C0000201F16B0401080E016F0401100E026F42
:1070D000040E036F04018C0E006F0401046B120098
:1070E0008B8E8986899454B0898492940000899605
:1070F00055A08994898655B08984569E899689863B
:1071000092848996898680B4568E89968B9E1200C9
:107110005438556E5638576E5AC05CF05BC05DF0FF
:10712000FE0E5A6E040E5B6E06EE00F0EE6AEAA6E4
:10713000FDD7120007EEFFF0BAD85CC05AF05DC070
:107140005BF08038ED125D6EEA8200D000D000D096
:107150000ED081AAA9D08038ED12EA825D6E551456
:1071600057181EE15C5058140EE1594EAAD08050B9
:10717000EF6E5C6E5414561816E15D385814E9E150
:10718000592EE9D7AAD000008050EF6E5C6E5414DF
:10719000561809E15D385814DCE1592EDCD79DD032
:1071A00081AA82D0E4D70000D4D707EEFFF07FD8C1
:1071B0005CC05AF05DC05BF08038ED125D6EEA8213
:1071C00000D000D000D00ED081AA6ED08038ED1251
:1071D000EA825D6E551457181EE15C5058140EE09B
:1071E000594E6FD08050EF6E5C6E5414561816E1F5
:1071F0005D385814E9E0592EE9D76FD0000080506F
:10720000EF6E5C6E5414561809E15D385814DCE0DA
:10721000592EDCD762D081AA47D0E4D70000D4D75A
:1072200007EEFFF044D85CC05AF05DC05BF07DD83B
:1072300000008038ED125D6EEA8200D000D000D0F0
:10724000000010D081AA30D070D88038ED12EA82C8
:107250005D6E5514571823E15C5058145F1810E107
:10726000594E2FD062D88050EF6E5C6E5414561871
:1072700019E15D3858145F18E5E1592EE5D72DD096
:10728000000053D88050EF6E5C6E541456180AE11B
:107290005D3858145F18D6E1592ED6D71ED081AA72
:1072A00003D0E0D700D0CED7400E556E12008050EC
:1072B000EF6E00D000D000D000005E5227E035D83D
:1072C00025D08050EF6EE9CF54F0EA508009556E1A
:1072D00000D05E521BE029D819D08038ED12EA8226
:1072E000E9CF54F0EACF55F000D05E5202E01DD84D
:1072F00000D08050EF6E00005A2E15D05B4E120069
:10730000000000005E5202E010D800D08038ED127C
:10731000EA825A2E09D05B4E1200000000005E5235
:10732000E8E003D8E6D7EDD7F9D75E5000D000D01B
:107330000000E84E120000D00000F8D7000EF36EF7
:1073400000EE00F0040E01D81200EA6002D0EE6AEE
:10735000FCD7F350E9601200EE6AFCD7040110512B
:107360001F0B010801E07DD00401145101E079D028
:10737000060E0401115D2FE104011351230A28E0D8
:10738000010A13E0030A01E024D00201020EF26FA9
:107390000001EF0505E10201680EF36F7A0EF46F4C
:1073A000090E0201F76FF86B14D00201020EF26FA2
:1073B0000001EF0505E102011F0EF36F7B0EF46F74
:1073C0000001EF0504E11D0E0201F76FF86B01D01B
:1073D00000D00001EE8304011051600BE842E84246
:1073E000E842E842E842010801E03BD004011151C3
:1073F0000B0A31E0080A21E0090A19E0080A09E04D
:107400000B0A05E0080A01E02CD02CD82AD02BD892
:1074100028D00201020EF26F0201F10EF36F000E8E
:10742000F46F0001EE930201010EF76F1AD0020112
:10743000020EF26F13C4F1F014D00201020EF26FCB
:107440000201F20EF36F000EF46F0001EE930201E1
:10745000010EF76F06D00201020EF26F12C4F2F0B5
:1074600000D01200120012000001F36B1E0E716EAC
:107470000401400E096F0401200E0A6F040E0B6F09
:107480000401880E086F0401600E0E6F040E0F6F6A
:107490000401400E0C6F1200D9CFE6FFE1CFD9FFF7
:1074A000E652FC0EDB50400805E2400EF36EFC0E87
:1074B000F3CFDBFFDF6AFC0EDB50DF5C19E2DF504D
:1074C000E76EFD0EDBCFE9FFFE0EDBCFEAFFE750F4
:1074D000E926000EEA22EF50E66EDF50EA6A600FFE
:1074E000E96E040EEA22E552E750EF6EDF2AE3D799
:1074F000FC0EDBCF0DF4400E04010C1704010C7DD3
:10750000880E04010C13E552E552E7CFD9FF1200B3
:10751000D9CFE6FFE1CFD9FF0001F36B040108BF2B
:1075200039D0FC0EDBCF3FF004010951D8803F5425
:1075300003E2FC0E09C4DBFF0001F36BFC0EDB5021
:107540000001F35D1CE20001F351EA6A200FE96ECD
:10755000040EEA22EF50E66E0001F351E76EFD0ED5
:10756000DBCFE9FFFE0EDBCFEAFFE750E926000E96
:10757000EA22E552E750EF6E0001F32BDFD704015A
:10758000400E096F400E040108170401087D880EA3
:10759000040108130001F35100D0E552E7CFD9FFF1
:1075A0001200D8CFE4FFE0CFE4FFE46EDACFE4FFCF
:1075B000E2CFDAFFE6520001E8A37CD0A150400BF5
:1075C0001DE0A050400B1AE0B4BE17D0A09CCD988F
:1075D0003550CF6E480E3424496E4A6A000E4A2256
:1075E0004A3404E24950FF08000E4A5401E2CF2A0F
:1075F000480E3424CE6E9E909D80A19C9E50010B1F
:1076000031E09D50010B2EE03550CF6E3450CE6EE0
:107610009E9036500AE1CD88B4AE04D09D90A19CD6
:10762000A08C02D08B80362A1DD03650080815E277
:10763000B4AE0DD03DA003D037503B6E07D03DA275
:1076400003D037503C6E02D037503A6E3D2A8B90B3
:10765000366A9D90A19CA08C05D037903742B4BE6D
:10766000378E362AA150020B24E0A050020B21E0F5
:107670003550B36E3450B26EA192385004E1899601
:10768000382A8B8016D0090E385C03E18986382AA7
:1076900010D03850090804E2386AA0928B9009D0C3
:1076A000010E3914E8B08986E8A08996382A399005
:1076B000394262D09EA035D09E90FA0ECF6E380E21
:1076C000CE6E8150100B10E10201FA51C45C0CE245
:1076D0000C0E0201FC5D05E18A948A880001E789AD
:1076E00002D00201FC2B02D00201FC6B300E000123
:1076F000E71512E00201FEC249F0FFC24AF0FE2B7C
:10770000000EFF239B0ED8804954020E4A5404E217
:107710008B700201FE6BFF6B9E9C010EC26E9D8CF6
:10772000C2829EAC29D09E9C0C0EBA5C21E1000165
:10773000E151D880C45401E2BB6A0001E251C45C4B
:1077400002E2E0C0BBFF8150040B10E00201FB51DC
:10775000C45C0CE20C0E0201FD5D05E18A948A888E
:107760000001E78B02D00201FD2B02D00201FD6B6C
:10777000050EC26E9D9CC282A1B4FF00E552E5CF0A
:10778000DAFFE550E5CFE0FFE5CFD8FF10000201BA
:10779000FC6B0201FD6B800ECD6EFA0ECF6E380EC3
:1077A000CE6E9E909D80CD809E9C9D9C260EC06E30
:1077B000050EC26EC28212009D90CD90C26A9E9C40
:1077C0009D9C120004011051600BE842E842E8421F
:1077D000E842E842000901E0A0D004011151080A82
:1077E00001E18CD0010A01E177D00F0A0AE0030A17
:1077F00001E092D00201010EF26F0001040EED6F64
:107800008CD00201010EF26F040113050AE102019E
:10781000440EF36F7A0EF46F120E0201F76FF86BDD
:1078200058D0020E0401135D1FE104011251F66EDF
:10783000F76AD890F636F7363C0EF6267B0EF7221E
:107840000900F5CFF3F20A00F5CFF4F2020E0201BF
:10785000F76AF325F66EF451F7220900F5CFF7F237
:107860000A00F5CFF8F235D0030E0401135D2FE1C5
:10787000030E0401125D10E10201000EF36F000E11
:10788000F46FF3C2E9FFF4C2EAFFEF500201F76FB1
:10789000F86B0001EE9341D004011251F66EF76AC5
:1078A000D890F636F736400EF6267B0EF722090002
:1078B000F5CFF3F20A00F5CFF4F2F3C2F6FFF4C20B
:1078C000F7FF0800F5500201F76FF86B02D00201D4
:1078D000F26B0001EE8321D00201010EF26F12C49F
:1078E000EFF00401125104E10001050EED6F05D027
:1078F0000001060EED6F34EC3AF00FD00201010EDC
:10790000F26F0201EF0EF36F000EF46F0001EE93C1
:107910000201010EF76F01D000D0120029C033F030
:1079200028C032F028502D02F4CF27F0F3CF26F0F4
:1079300029502E02F4CF29F0F3CF28F02D02F35076
:107940002726F4502822E86A292232502E02F350CA
:107950002726F4502822E86A29222EAEB4EF3CF004
:107960003250285E3350295A33AE000C2D50285E19
:107970002E50295A000C28C032F028502D02F4CF86
:1079800027F0F3CF26F029502E02F4CF29F0F3CFC1
:1079900028F02D02F3502726F4502822E86A2922E5
:1079A00032502E02F3502726F4502822E86A29226A
:1079B000000C29C033F028C032F027C031F0275026
:1079C0002C02F4CF25F0F3CF24F028502D02F4CF71
:1079D00027F0F3CF26F02C02F3502526F450262270
:1079E000E86A272231502D02F3502526F450262232
:1079F000E86A272229502C02F3502626F450272229
:107A000029502D02286AE86A2822F3502726F450CC
:107A1000282231502E02F3502626F4502722296ABC
:107A2000E86A2822292232502E02F3502726F450E9
:107A30002822E86A292233502E02F3502826F450D7
:107A40002922000C1201000200000008D8043300B3
:107A50000200010203020902290001010280F0096B
:107A60000400000203000000092101000001221DA2
:107A700000070581034000010705010340000109DB
:107A800002200001020480F00904000002FF00004F
:107A900000070581034000010705010340000104C0
:107AA00003090434034D006900630072006F006332
:107AB00000680069007000200054006500630068E1
:107AC000006E006F006C006F0067007900200049B5
:107AD000006E0063002E0048035000490043006B15
:107AE00000690074002000320020004D006900632E
:107AF0000072006F0063006F006E00740072006F10
:107B0000006C006C00650072002000500072006F75
:107B1000006700720061006D006D00650072000674
:107B200000FF0901A10119012940150026FF007578
:107B30000895408102190129409102C0567A7F7A46
:107B40009F7AA37AD77A5C73080E6D6E6DBAFED7F2
:107B5000686A110E696E0001020EED6F12006D6A07
:107B6000696A0001ED6B12006850040B09E069506E
:107B7000040B06E06D92699468A402D06894FCD767
:107B80006850010B04E06950010B01E025D86850F2
:107B9000200B06E06950200B03E070B07090689AEB
:107BA000030E0001ED5D01E216D00001F66B040E3C
:107BB0000001F65D10E26850080B09E06950080BFF
:107BC00006E0B9EC36F0000901E1689601D003D077
:107BD0000001F62BECD71200686A7B0E696E6E6AA4
:107BE000160E706E68A608D06896000000000000AF
:107BF000000000000000F6D76D9860EC38F000013E
:107C0000EF6B0001030EED6F1200000EF66E5C0EBE
:107C1000F76E000EF86E02010900F550EC6F0900D6
:107C2000F550ED6F03E1EC6701D03DD00900F55050
:107C3000E76F0900F550E86F0900F550E96F09009A
:107C40000900F550E96E0900F550EA6E09000900D7
:107C50000900F550EA6F0900F550EB6F09000900C3
:107C6000F6CFEEF2F7CFEFF2F8CFF0F2E7C2F6FF81
:107C7000E8C2F7FFE9C2F8FF0201EA5302E1EB5361
:107C800007E00900F550EE6EEA07F8E2EB07F9D7D6
:107C9000EEC2F6FFEFC2F7FFF0C2F8FF0201EC07F9
:107CA000000EED5BBFD7120026502B02F3CF22F05F
:107CB000F4CF23F02C02F3502326000EF420246E80
:107CC00026502D02F3502426000EF420256E265057
:107CD0002E02F350252627502B02F3502326F45072
:107CE0002422000E252227502C02F3502426F45083
:107CF000252227502D02F350252628502B02F35021
:107D00002426F450252228502C02F35025262950F1
:107D10002B02F35025261200FF0EE3504C6EEF0E9F
:107D200001D0F30EE76EE72E93EF3EF00C0E4B6E94
:107D3000E76AE72E99EF3EF04B2E98EF3EF04C2E7F
:107D400091EF3EF0120006D8B4EC3DF00BEC11F0D0
:107D5000FBD71200140E6F6E0001ED6B0001EE6B8D
:107D60000001EF6B15EC10F0A4EC3DF0120013EEE7
:107D700000F023EE00F0F86A219C05EC3EF0DEEC0A
:107D80003EF0A3EC3EF0FBD71200FF0EE3504C6E2A
:107D90001B0E00D001D0200EE76EE72EFED74C2E32
:107DA000FAD700D01200FF0EE350E84E1200000098
:107DB00000D000D000D0E82EFAD712001200000543
:107DC000FFFFFFFFFFFFFFFFFFFFFFFFFFFFFFFFC3
:107DD000FFFFFFFFFFFFFFFFFFFFFFFFFFFFFFFFB3
:107DE000FFFFFFFFFFFFFFFFFFFFFFFFFFFFFFFFA3
:107DF000FFFFFFFFFFFFFFFFFFFFFFFFFFFFFFFF93
:0200000400F00A
:020000040030CA
:0E000000240E361E008181000FC00EA00F409E
:020000040020DA
:08000000FFFFFFFFFFFFFFFF00
:00000001FF
